:020000040000FA
:0408000098EF0BF072
:1008100003B275EF05F0F2B493EF05F09EB09BEFD5
:1008200005F09EB2A3EF05F0F2A81AEF04F0F2B2C1
:1008300023EF04F0F2B01FEF04F047EF0BF0F29655
:10084000F29047EF0BF0CD90F2929EA02DEF04F0C6
:100850000101533F2DEF04F0542BB2C1B6F1B3C1E7
:10086000B7F1B4C1B8F1B5C1B9F1AEC1B2F1AFC120
:10087000B3F1B0C1B4F1B1C1B5F1AAC1AEF1ABC130
:10088000AFF1ACC1B0F1ADC1B1F1A6C1AAF1A7C140
:10089000ABF1A8C1ACF1A9C1ADF1A2C1A6F1A3C150
:1008A000A7F1A4C1A8F1A5C1A9F19EC1A2F19FC160
:1008B000A3F1A0C1A4F1A1C1A5F19AC19EF19BC170
:1008C0009FF19CC1A0F19DC1A1F1CECF9AF1CFCFF4
:1008D0009BF153C19CF154C19DF1CF6ACE6A0101D5
:1008E000536B546B9E90CD800FBC0F8E0FBA7CEF74
:1008F00004F00F8A47EF0BF013880F8C0FBEB9EF8F
:1009000004F09AC19EF19BC19FF19CC1A0F19DC1D1
:10091000A1F19EC1A2F19FC1A3F1A0C1A4F1A1C107
:10092000A5F1A2C1A6F1A3C1A7F1A4C1A8F1A5C1D7
:10093000A9F1A6C1AAF1A7C1ABF1A8C1ACF1A9C1A7
:10094000ADF1AAC1AEF1ABC1AFF1ACC1B0F1ADC177
:10095000B1F1AEC1B2F1AFC1B3F1B0C1B4F1B1C147
:10096000B5F1B2C1B6F1B3C1B7F1B4C1B8F1B5C117
:10097000B9F101015E6B5F6B606B616B9A515E2731
:100980009B515F239C5160239D5161239E515E27A3
:100990009F515F23A0516023A1516123A2515E2783
:1009A000A3515F23A4516023A5516123A6515E2763
:1009B000A7515F23A8516023A9516123AA515E2743
:1009C000AB515F23AC516023AD516123AE515E2723
:1009D000AF515F23B0516023B1516123B2515E2703
:1009E000B3515F23B4516023B5516123B6515E27E3
:1009F000B7515F23B8516023B9516123D8900101E9
:100A0000613360335F335E33D8900101613360330B
:100A10005F335E33D8900101613360335F335E33FF
:100A200000C10CF101C10DF102C10EF103C10FF1C2
:100A300004C110F105C111F106C112F107C113F192
:100A400008C114F109C115F10AC116F10BC117F162
:100A500034C135F111B838EF05F00101620E046FB1
:100A6000010E056F000E066F000E076F41EF05F0D7
:100A70000101A70E046F020E056F000E066F000E37
:100A8000076F5EC100F15FC101F160C102F161C198
:100A900003F1D9EC2FF003BF04D01CBE02D01CA080
:100AA000108C11A059EF05F010BA59EF05F00F8026
:100AB000108A0CC100F10DC101F10EC102F10FC18C
:100AC00003F110C104F111C105F112C106F113C106
:100AD00007F114C108F115C109F116C10AF117C1D6
:100AE0000BF135C134F147EF0BF00392ABB2AB9889
:100AF000AB88030103EE00F080517F0BE92604C0B0
:100B0000EFFF802B8151805D700BD8A48B82000099
:100B10008051815D700BD8A48B9281518019D8B41B
:100B2000079047EF0BF0F2940101453F47EF0BF0C0
:100B3000462B47EF0BF09E900101533F47EF0BF020
:100B4000542B47EF0BF09E9211B843EF08F00400CE
:100B500066A1ABEF05F08BB4B5EF05F010ACB5EFC7
:100B600005F08B84109CB6EF05F08B94077C07ACE6
:100B7000D1EF05F0C274C2B4CBEF05F0C3CFB7F527
:100B8000C4CFB8F50501D890B833B733D890B8338F
:100B9000B733D2EF05F0C3CF55F1C4CF56F1D2EF42
:100BA00005F0C28207B444EF06F047C14BF148C1DB
:100BB0004CF149C14DF14AC14EF15EC162F15FC1D4
:100BC00063F160C164F161C165F113A8EAEF05F05A
:100BD000138C13989AC1BAF19BC1BBF19CC1BCF1B3
:100BE0009DC1BDF19EC1BEF19FC1BFF1A0C1C0F1C9
:100BF000A1C1C1F1A2C1C2F1A3C1C3F1A4C1C4F199
:100C0000A5C1C5F1A6C1C6F1A7C1C7F1A8C1C8F168
:100C1000A9C1C9F1AAC1CAF1ABC1CBF1ACC1CCF138
:100C2000ADC1CDF1AEC1CEF1AFC1CFF1B0C1D0F108
:100C3000B1C1D1F1B2C1D2F1B3C1D3F1B4C1D4F1D8
:100C4000B5C1D5F1B6C1D6F1B7C1D7F1B8C1D8F1A8
:100C5000B9C1D9F1B7C5B9F5B8C5BAF5B9C5BBF5CC
:100C6000BAC5BCF5010155515B2756515C23E86AB2
:100C70005D230E2E44EF06F05CC157F15DC158F1C3
:100C80005B6B5C6B5D6B078E0201002F47EF0BF017
:100C90003C0E006F1D50E00BE00AE86612881BBE98
:100CA00002D01BB4108E00C10CF101C10DF102C1C4
:100CB0000EF103C10FF104C110F105C111F106C11C
:100CC00012F107C113F108C114F109C115F10AC1EC
:100CD00016F10BC117F134C135F181AAACEF06F062
:100CE00015A4F7EF06F005012F51000AD8B43AEF2A
:100CF00007F005012F51010AD8B4B6EF06F005013F
:100D00002F51020AD8B4F7EF06F005012F51030A5C
:100D1000D8B4F7EF06F005012F51040AD8B4F7EF65
:100D200006F005012F51050AD8B4F7EF06F00501CA
:100D30002F51060AD8B4F7EF06F005012F51070A24
:100D4000D8B4F7EF06F005012F51320AD8B4B4EF4A
:100D500006F02F6B3AEF07F000011650030AD8B4E3
:100D6000F7EF06F03AEF07F03AEF07F005015767A3
:100D7000C1EF06F05867C1EF06F05967C1EF06F002
:100D80005A67C5EF06F03AEF07F05BC500F15CC5A6
:100D900001F15DC502F15EC503F10101010E046FB1
:100DA000000E056F000E066F000E076FD9EC2FF0D6
:100DB00000C15BF501C15CF502C15DF503C15EF5E3
:100DC00001010067EBEF06F00167EBEF06F0026749
:100DD000EBEF06F003673AEF07F057C55BF558C530
:100DE0005CF559C55DF55AC55EF524EF07F00FBEF9
:100DF0000CEF07F010A011EF07F00101476708EFB3
:100E000007F0486708EF07F0496708EF07F04A67FF
:100E10000CEF07F011EF07F007AE11EF07F024EF2A
:100E200007F00501312F3AEF07F03C0E316F302FFC
:100E30003AEF07F00101000E626FE00E636FA50E3E
:100E4000646F010E656F138800011650000AD8B454
:100E500032EF07F000011650030AD8B437EF07F05D
:100E60003AEF07F00001010E166E3AEF07F00001AD
:100E7000040E166E0501666B37B740EF07F066810A
:100E80000CC100F10DC101F10EC102F10FC103F15E
:100E900010C104F111C105F112C106F113C107F12E
:100EA00014C108F115C109F116C10AF117C10BF1FE
:100EB00035C134F100C10CF101C10DF102C10EF1D7
:100EC00003C10FF104C110F105C111F106C112F106
:100ED00007C113F108C114F109C115F10AC116F1D6
:100EE0000BC117F134C135F101018E677FEF07F0B7
:100EF0008F677FEF07F090677FEF07F0916783EFD1
:100F000007F0B4EF07F092C100F193C101F194C171
:100F100002F195C103F10101010E046F000E056F8E
:100F2000000E066F000E076FD9EC2FF000C192F192
:100F300001C193F102C194F103C195F10101006770
:100F4000A9EF07F00167A9EF07F00267A9EF07F023
:100F50000367B4EF07F08EC192F18FC193F190C196
:100F600094F191C195F10F80D57ED5BE6ED0D6CFCC
:100F700047F1D7CF48F145C149F1E86AE8CF4AF1D6
:100F8000138A1CBE02D01CA0108C109047C100F127
:100F900048C101F149C102F14AC103F101010A0E40
:100FA000046F000E056F000E066F000E076FD9EC80
:100FB0002FF003AF1080010154A7EBEF07F00F9A59
:100FC0000F9C0F9E0101000E5E6F600E5F6F3D0E65
:100FD000606F080E616F010147BFFBEF07F04867C4
:100FE000FBEF07F04967FBEF07F04A67FBEF07F0FD
:100FF000F28820EF08F0F2985E6B5F6B606B616BBC
:101000009A6B9B6B9C6B9D6B9E6B9F6BA06BA16B9C
:10101000A26BA36BA46BA56BA66BA76BA86BA96B4C
:10102000AA6BAB6BAC6BAD6BAE6BAF6BB06BB16BFC
:10103000B26BB36BB46BB56BB66BB76BB86BB96BAC
:10104000D76AD66A0101456B466B0CC100F10DC130
:1010500001F10EC102F10FC103F110C104F111C180
:1010600005F112C106F113C107F114C108F115C150
:1010700009F116C10AF117C10BF135C134F147EF7F
:101080000BF047EF0BF00201002FABEF0AF0D59EFB
:10109000D6CF47F1D7CF48F145C149F1E86AE8CF4B
:1010A0004AF1138AD76AD66A0101456B466BD58E21
:1010B0001D50E00BE00AE86612881BBE02D01BB48C
:1010C000108E1AAE1F8C00C10CF101C10DF102C1CE
:1010D0000EF103C10FF104C110F105C111F106C1F8
:1010E00012F107C113F108C114F109C115F10AC1C8
:1010F00016F10BC117F134C135F10FA0109A11B8D8
:101100008DEF08F00101620E046F010E056F000EF5
:10111000066F000E076F96EF08F00101A70E046F2F
:10112000020E056F000E066F000E076F47C100F13B
:1011300048C101F149C102F14AC103F1D9EC2FF0D4
:1011400003BFA9EF08F01CBE02D01CA0108C11B088
:101150000F800CC100F10DC101F10EC102F10FC1F0
:1011600003F110C104F111C105F112C106F113C15F
:1011700007F114C108F115C109F116C10AF117C12F
:101180000BF135C134F102013C0E006F00C10CF1CE
:1011900001C10DF102C10EF103C10FF104C110F143
:1011A00005C111F106C112F107C113F108C114F113
:1011B00009C115F10AC116F10BC117F134C135F19E
:1011C00081BAE6EF08F015B225EF09F015A025EF7A
:1011D00009F015A470EF09F005012F51000AD8B4E9
:1011E000B3EF09F005012F51010AD8B42FEF09F030
:1011F00005012F51020AD8B470EF09F005012F51F3
:10120000030AD8B470EF09F005012F51040AD8B4CD
:1012100070EF09F005012F51050AD8B470EF09F0FD
:1012200005012F51060AD8B470EF09F005012F51BE
:10123000070AD8B470EF09F005012F51320AD8B46B
:101240002DEF09F02F6BB3EF09F000011650030AE0
:10125000D8B470EF09F0B3EF09F0B3EF09F005016E
:1012600057673AEF09F058673AEF09F059673AEFD4
:1012700009F05A673EEF09F0B3EF09F05BC500F1E2
:101280005CC501F15DC502F15EC503F10101010E0E
:10129000046F000E056F000E066F000E076FD9EC8D
:1012A0002FF000C15BF501C15CF502C15DF503C122
:1012B0005EF50101006764EF09F0016764EF09F072
:1012C000026764EF09F00367B3EF09F057C55BF5F8
:1012D00058C55CF559C55DF55AC55EF59DEF09F039
:1012E0000FBE85EF09F010A08AEF09F001014767F2
:1012F00081EF09F0486781EF09F0496781EF09F054
:101300004A6785EF09F08AEF09F007AE8AEF09F026
:101310009DEF09F00501312FB3EF09F03C0E316F5D
:10132000302FB3EF09F00101000E626FE00E636F22
:10133000A50E646F010E656F138800011650000A38
:10134000D8B4ABEF09F000011650030AD8B4B0EFDF
:1013500009F0B3EF09F00001010E166EB3EF09F0CA
:101360000001040E166E0501666B37B7B9EF09F080
:1013700066810CC100F10DC101F10EC102F10FC176
:1013800003F110C104F111C105F112C106F113C13D
:1013900007F114C108F115C109F116C10AF117C10D
:1013A0000BF135C134F100C10CF101C10DF102C1E5
:1013B0000EF103C10FF104C110F105C111F106C115
:1013C00012F107C113F108C114F109C115F10AC1E5
:1013D00016F10BC117F134C135F101018E67F8EF39
:1013E00009F08F67F8EF09F09067F8EF09F091675F
:1013F000FCEF09F02DEF0AF092C100F193C101F169
:1014000094C102F195C103F10101010E046F000EB8
:10141000056F000E066F000E076FD9EC2FF000C1AC
:1014200092F101C193F102C194F103C195F101015F
:10143000006722EF0AF0016722EF0AF0026722EF4D
:101440000AF003672DEF0AF08EC192F18FC193F17C
:1014500090C194F191C195F10F80109047C100F1B6
:1014600048C101F149C102F14AC103F101010A0E6B
:10147000046F000E056F000E066F000E076FD9ECAB
:101480002FF003AF1080010154A753EF0AF00F9A19
:101490000F9C0F9E0101000E5E6F600E5F6F3D0E90
:1014A000606F080E616F47C100F148C101F149C189
:1014B00002F14AC103F10101140E046F050E056F1C
:1014C000000E066F000E076FD9EC2FF003AF6CEF24
:1014D0000AF0F28891EF0AF0F2985E6B5F6B606B36
:1014E000616B9A6B9B6B9C6B9D6B9E6B9F6BA06BF8
:1014F000A16BA26BA36BA46BA56BA66BA76BA86B70
:10150000A96BAA6BAB6BAC6BAD6BAE6BAF6BB06B1F
:10151000B16BB26BB36BB46BB56BB66BB76BB86BCF
:10152000B96B0CC100F10DC101F10EC102F10FC187
:1015300003F110C104F111C105F112C106F113C18B
:1015400007F114C108F115C109F116C10AF117C15B
:101550000BF135C134F104008BB4B6EF0AF010ACD6
:10156000B6EF0AF08B84109CB7EF0AF08B94077CDF
:1015700007ACD2EF0AF0C274C2B4CCEF0AF0C3CF0A
:10158000B7F5C4CFB8F50501D890B833B733D890C4
:10159000B833B733D3EF0AF0C3CF55F1C4CF56F108
:1015A000D3EF0AF0C28207B445EF0BF047C14BF10D
:1015B00048C14CF149C14DF14AC14EF15EC162F1E1
:1015C0005FC163F160C164F161C165F113A8EBEF24
:1015D0000AF0138C13989AC1BAF19BC1BBF19CC15C
:1015E000BCF19DC1BDF19EC1BEF19FC1BFF1A0C1C3
:1015F000C0F1A1C1C1F1A2C1C2F1A3C1C3F1A4C193
:10160000C4F1A5C1C5F1A6C1C6F1A7C1C7F1A8C162
:10161000C8F1A9C1C9F1AAC1CAF1ABC1CBF1ACC132
:10162000CCF1ADC1CDF1AEC1CEF1AFC1CFF1B0C102
:10163000D0F1B1C1D1F1B2C1D2F1B3C1D3F1B4C1D2
:10164000D4F1B5C1D5F1B6C1D6F1B7C1D7F1B8C1A2
:10165000D8F1B9C1D9F1B7C5B9F5B8C5BAF5B9C5A9
:10166000BBF5BAC5BCF5010155515B2756515C234A
:10167000E86A5D230E2E45EF0BF05CC157F15DC1AA
:1016800058F15B6B5C6B5D6B078E47EF0BF002C034
:10169000E0FF005001C0D8FF1000A6B24DEF0BF0E4
:1016A0000CC0A9FF0BC0A8FFA69EA69CA684F29E14
:1016B000550EA76EAA0EA76EA682F28EA694A6B2AB
:1016C0005FEF0BF00C2A1200A96EA69EA69CA680C6
:1016D000A8500C2A120004012C0E826F96EC0EF01A
:1016E000EEEC30F00C5064EC0BF0E8CF00F10C5055
:1016F00064EC0BF0E8CF01F101AF84EF0BF00101D6
:10170000FF0E026FFF0E036F77EC30F0296790EF4A
:101710000BF00401200E826F96EC0EF095EF0BF0AB
:1017200004012D0E826F96EC0EF081EC2EF012006B
:1017300015941596076A0F6A106A116A126A136A7D
:10174000166A0F010D0EC16E860EC06E030EC26EBC
:101750000F01680E896E130E926E080E8A6EF30EDC
:10176000936E8B6A900E946EC80E64EC0BF0E8CF0B
:10177000E8FF1098E8A0108810A805D00E0E256E7E
:101780008E0E266E04D00F0E256E8F0E266E86EC02
:1017900031F0D1EC32F0F18EF19EFC0E64EC0BF0E6
:1017A000E8CF0BF00BA011800BA211820BA41184C7
:1017B0000BA81188C90E64EC0BF0E8CF1AF0CA0E22
:1017C00064EC0BF0E8CF1BF0CB0E64EC0BF0E8CF31
:1017D0001CF0CC0E64EC0BF0E8CF1DF0FB0E64ECBB
:1017E0000BF0E8CF37F0CE0E64EC0BF0E8CF14F03E
:1017F000CD0E64EC0BF0E8CF36F01F6A206A0E6A5B
:1018000001015B6B5C6B5D6B576B586BF29A01016E
:10181000476B486B496B4A6B4B6B4C6B4D6B4E6B1C
:101820004F6B506B516B526B456B466BD76AD66AE8
:101830000F01280ED56EF28A9D90B00ECD6E01017B
:101840005E6B5F6B606B616B626B636B646B656B34
:10185000666B676B686B696B536B546BCF6ACE6A50
:101860000F9A0F9C0F9E9D80760ECA6E9D8202017C
:101870003C0E006FCC6A160E64EC0BF0E8CF00F162
:10188000170E64EC0BF0E8CF01F1180E64EC0BF0CE
:10189000E8CF02F1190E64EC0BF0E8CF03F101017F
:1018A00003AF6DEF0CF0EEEC30F0160E0C6E00C1D5
:1018B0000BF04DEC0BF0170E0C6E01C10BF04DEC64
:1018C0000BF0180E0C6E02C10BF04DEC0BF0190E64
:1018D0000C6E03C10BF04DEC0BF000C18EF101C199
:1018E0008FF102C190F103C191F100C192F101C1E8
:1018F00093F102C194F103C195F11A0E64EC0BF05F
:10190000E8CF00F11B0E64EC0BF0E8CF01F11C0EE8
:1019100064EC0BF0E8CF02F11D0E64EC0BF0E8CFA5
:1019200003F1010103AFC3EF0CF0EEEC30F01A0E3F
:101930000C6E00C10BF04DEC0BF01B0E0C6E01C1D8
:101940000BF04DEC0BF01C0E0C6E02C10BF04DECCD
:101950000BF01D0E0C6E03C10BF04DEC0BF01A0ECC
:1019600064EC0BF0E8CF00F11B0E64EC0BF0E8CF59
:1019700001F11C0E64EC0BF0E8CF02F11D0E64ECDB
:101980000BF0E8CF03F100C196F101C197F102C15C
:1019900098F103C199F1240EAC6E900EAB6E240E3B
:1019A000AC6E080EB86E000EB06E1F0EAF6E040166
:1019B000806B816B0F01900EAB6E0F019D8A03014E
:1019C000806B816BC26B8B922BEC36F02BEC36F07C
:1019D0000DEC38F009EC34F0200E64EC0BF0E8CF9D
:1019E0002FF505012F51FF0AD8A4FEEF0CF02F6B45
:1019F000200E0C6E2FC50BF04DEC0BF00501010E07
:101A0000306F3C0E316F250E64EC0BF0E8CF00F127
:101A1000260E64EC0BF0E8CF01F1270E64EC0BF01E
:101A2000E8CF02F1280E64EC0BF0E8CF03F10101DE
:101A300003AF35EF0DF0EEEC30F0250E0C6E00C16B
:101A40000BF04DEC0BF0260E0C6E01C10BF04DECC3
:101A50000BF0270E0C6E02C10BF04DEC0BF0280EB4
:101A60000C6E03C10BF04DEC0BF000C157F501C13A
:101A700058F502C159F503C15AF500C15BF501C122
:101A80005CF502C15DF503C15EF5290E64EC0BF057
:101A9000E8CF5FF5050160515F5DD8A05FC560F5D7
:101AA000210E64EC0BF0E8CF00F1220E64EC0BF099
:101AB000E8CF01F1230E64EC0BF0E8CF02F1240E25
:101AC00064EC0BF0E8CF03F1010103AF96EF0DF0EA
:101AD000EEEC30F0210E0C6E00C10BF04DEC0BF073
:101AE000220E0C6E01C10BF04DEC0BF0230E0C6EB0
:101AF00002C10BF04DEC0BF0240E0C6E03C10BF089
:101B00004DEC0BF0210E64EC0BF0E8CF00F1220E4F
:101B100064EC0BF0E8CF01F1230E64EC0BF0E8CF9E
:101B200002F1240E64EC0BF0E8CF03F100C161F583
:101B300001C162F502C163F503C164F551EC33F0F4
:101B400037EC32F08FEC31F01590C70E64EC0BF0EF
:101B5000E8CF00F1010100B1B1EF0DF01592B2EF45
:101B60000DF0158281AAC0EF0DF015B4BBEF0DF09A
:101B70001580C0EF0DF04CEC38F015A0B3EF38F045
:101B800007900001F28EF28C12AE03D012BC6EEF01
:101B900019F007B000EF2DF00FB0A8EF25F010BE40
:101BA000A8EF25F012B8A8EF25F000011650010AA1
:101BB000D8B4A1EF1DF081BAE6EF0DF00001165088
:101BC000040AD8B41AEF1CF0ECEF0DF00001165027
:101BD000040AD8B4DDEF1DF00301805181197F0B99
:101BE000D8B400EF2DF013EE00F081517F0BE12609
:101BF000812BE7CFE8FFE00BD8B400EF2DF023EE08
:101C000082F0C2513F0BD926E7CFDFFFC22BDF5056
:101C1000780AD8A400EF2DF0078092C100F193C19B
:101C200001F194C102F195C103F10101040E046FA9
:101C3000000E056F000E066F000E076FD9EC2FF037
:101C400000AF2CEF0EF00101030E926F000E936FA8
:101C5000000E946F000E956F03018251720AD8B482
:101C600029EF25F08251520AD8B429EF25F082518C
:101C7000750AD8B429EF25F08251680AD8B4AAEFC2
:101C80000EF08251630AD8B4BAEF29F08251690A82
:101C9000D8B4E7EF20F082517A0AD8B4FAEF21F0F5
:101CA0008251490AD8B486EF20F08251500AD8B444
:101CB000A4EF1FF08251700AD8B4E7EF1FF08251F1
:101CC000540AD8B412EF20F08251740AD8B458EFF5
:101CD00020F08251410AD8B4AFEF0FF082514B0A85
:101CE000D8B4ACEF0EF082516D0AD8B41FEF14F0E7
:101CF00082514D0AD8B438EF14F08251730AD8B427
:101D000059EF24F08251530AD8B4BEEF24F0825127
:101D10004C0AD8B4C7EF14F08251590AD8B470EF06
:101D200013F012AE01D0128CF1EF29F0040114EE81
:101D300000F080517F0BE12682C4E7FF802B120068
:101D400004010D0E826F96EC0EF00A0E826F96EC77
:101D50000EF01200EFEF29F004014B0E826F96ECAB
:101D60000EF004012C0E826F96EC0EF081B802D0BA
:101D700036B630D003018351430AD8B4F1EF0EF0E8
:101D800003018351630AD8B4F3EF0EF003018351CA
:101D9000520AD8B4F5EF0EF003018351720AD8B499
:101DA000F7EF0EF003018351470AD8B4F9EF0EF0B4
:101DB00003018351670AD8B4FBEF0EF0030183518E
:101DC000540AD8B4FDEF0EF003018351740AD8B45D
:101DD0006DEF0FF003018351550AD8B4FFEF0EF0F9
:101DE00083D036807BD0369079D0368277D03692C9
:101DF00075D0368473D0369471D036866FD084C354
:101E000030F185C331F186C332F187C333F101016B
:101E1000296B3CEC31F0B3EC30F000C104F101C1AE
:101E200005F102C106F103C107F12FEC31F0200EDC
:101E3000F86EF76AF66A0900F5CF2CF10900F5CFC4
:101E40002DF10900F5CF2EF10900F5CF2FF1090092
:101E5000F5CF30F10900F5CF31F10900F5CF32F1BE
:101E60000900F5CF33F10101296B3CEC31F0B3EC03
:101E700030F0D9EC2FF00101006746EF0FF0016759
:101E800046EF0FF0026746EF0FF0036701D025D051
:101E900004014E0E826F96EC0EF004016F0E826FFD
:101EA00096EC0EF004014D0E826F96EC0EF00401DC
:101EB000610E826F96EC0EF00401740E826F96EC48
:101EC0000EF00401630E826F96EC0EF00401680EB2
:101ED000826F96EC0EF0EFEF29F03696CD0E0C6E79
:101EE00036C00BF04DEC0BF0CD0E64EC0BF0E8CFF0
:101EF00036F036B006D00401630E826F96EC0EF019
:101F000005D00401430E826F96EC0EF036B206D077
:101F10000401720E826F96EC0EF005D00401520E91
:101F2000826F96EC0EF036B406D00401670E826F15
:101F300096EC0EF005D00401470E826F96EC0EF081
:101F400036B606D00401740E826F96EC0EF005D002
:101F50000401540E826F96EC0EF0EFEF29F00401AD
:101F6000410E826F96EC0EF003018351310AD8B412
:101F700090EF12F003018351320AD8B4C0EF11F090
:101F800003018351330AD8B449EF11F0030183519F
:101F9000340AD8B439EF10F003018351350AD8B4AC
:101FA000D9EF0FF004013F0E826F96EC0EF0EFEFC9
:101FB00029F003018451300AD8B4FFEF0FF0030178
:101FC0008451310AD8B402EF10F003018451650A3C
:101FD000D8B4F3EF0FF003018451640AD8B4F6EFDC
:101FE0000FF003EF10F03790F7EF0FF03780FB0E94
:101FF0000C6E37C00BF04DEC0BF003EF10F08B9034
:1020000003EF10F08B800401350E826F96EC0EF01A
:1020100004012C0E826F96EC0EF08BB017EF10F0CF
:102020000401300E826F96EC0EF01CEF10F00401EC
:10203000310E826F96EC0EF004012C0E826F96EC3E
:102040000EF0FB0E64EC0BF0E8CF37F037A030EF6A
:1020500010F00401640E826F96EC0EF035EF10F074
:102060000401650E826F96EC0EF037EF10F0EFEF83
:1020700029F0CC0E64EC0BF0E8CF0BF004012C0E31
:10208000826F96EC0EF003018451310AD8B45DEFF3
:1020900010F003018451300AD8B45FEF10F003014F
:1020A00084514D0AD8B469EF10F003018451540AE9
:1020B000D8B470EF10F087EF10F08A8401D08A94C2
:1020C0000BAE04D00BAC02D00BBA21D0E00E0B1239
:1020D00018D01F0E0B168539E844E00B0B1211D0F7
:1020E000E00E0B162FEC31F085C332F186C333F1CD
:1020F0000101296B3CEC31F0B3EC30F000511F0BC7
:102100000B12CC0E0C6E0BC00BF04DEC0BF004015F
:10211000340E826F96EC0EF004012C0E826F96EC5A
:102120000EF0CC0E64EC0BF0E8CF1DF08AB406D0B4
:102130000401300E826F96EC0EF005D00401310ED2
:10214000826F96EC0EF004012C0E826F96EC0EF06E
:102150001D38E840070BE8CF82F40401300E8227D7
:1021600096EC0EF004012C0E826F96EC0EF0EEEC65
:1021700030F01D501F0BE8CF00F177EC30F032C18A
:1021800082F40401300E822796EC0EF033C182F403
:102190000401300E822796EC0EF004012C0E826FA3
:1021A00096EC0EF0EEEC30F030C000F100AF0BD04A
:1021B000FF0E016FFF0E026FFF0E036F04012D0E65
:1021C000826F96EC0EF077EC30F031C182F40401AE
:1021D000300E822796EC0EF032C182F40401300EEC
:1021E000822796EC0EF033C182F40401300E822770
:1021F00096EC0EF004012C0E826F96EC0EF0EEECD5
:1022000030F02FC000F177EC30F031C182F40401DE
:10221000300E822796EC0EF032C182F40401300EAB
:10222000822796EC0EF033C182F40401300E82272F
:1022300096EC0EF004012C0E826F96EC0EF0EEEC94
:1022400030F031C000F100AF0BD0FF0E016FFF0E78
:10225000026FFF0E036F04012D0E826F96EC0EF0DD
:1022600077EC30F031C182F40401300E822796EC15
:102270000EF032C182F40401300E822796EC0EF08B
:1022800033C182F40401300E822796EC0EF0EFEF9A
:1022900029F0CB0E64EC0BF0E8CF0BF004012C0E10
:1022A000826F96EC0EF003018451450AD8B46DEFAD
:1022B00011F003018451440AD8B470EF11F0030106
:1022C0008451300AD8B473EF11F003018451310AFC
:1022D000D8B477EF11F082EF11F00B9E7CEF11F084
:1022E0000B8E7CEF11F0FC0E0B167CEF11F0FC0E48
:1022F0000B160B807CEF11F0CB0E0C6E0BC00BF0AD
:102300004DEC0BF00401330E826F96EC0EF00401DD
:102310002C0E826F96EC0EF0CB0E64EC0BF0E8CF37
:102320001CF01CBE9BEF11F00401450E826F96EC71
:102330000EF0A0EF11F00401440E826F96EC0EF047
:1023400004012C0E826F96EC0EF00401300E826FA9
:1023500096EC0EF004012C0E826F96EC0EF01CB081
:10236000B9EF11F00401300E826F96EC0EF0BEEF63
:1023700011F00401310E826F96EC0EF0EFEF29F0B0
:10238000CA0E64EC0BF0E8CF0BF004012C0E826F48
:1023900096EC0EF003018451450AD8B4FCEF11F01D
:1023A00003018451440AD8B4FFEF11F003018451B2
:1023B0004D0AD8B408EF12F003018451410AD8B491
:1023C00002EF12F003018451460AD8B405EF12F06F
:1023D00003018451560AD8B410EF12F0030184515E
:1023E000500AD8B41BEF12F003018451520AD8B43A
:1023F0001EEF12F027EF12F00B9E21EF12F00B8E62
:1024000021EF12F00B9C21EF12F00B8C21EF12F058
:10241000FC0E0B1685C3E8FF030B0B1221EF12F025
:10242000C70E0B1685C3E8FF070BE846E846E846EB
:102430000B1221EF12F00B8421EF12F00B9421EF1D
:1024400012F0CA0E0C6E0BC00BF04DEC0BF0CA0E66
:1024500064EC0BF0E8CF1BF00401320E826F96ECB7
:102460000EF004012C0E826F96EC0EF01BBE40EFB6
:1024700012F00401450E826F96EC0EF045EF12F05B
:102480000401440E826F96EC0EF004012C0E826F54
:1024900096EC0EF01BC0E8FF030BE8CF82F40401BA
:1024A000300E822796EC0EF004012C0E826F96EC13
:1024B0000EF01BBC63EF12F00401410E826F96EC2C
:1024C0000EF068EF12F00401460E826F96EC0EF0EB
:1024D00004012C0E826F96EC0EF01BC0E8FF380B47
:1024E000E842E842E842E8CF82F40401300E822755
:1024F00096EC0EF004012C0E826F96EC0EF01BB4DD
:1025000089EF12F00401520E826F96EC0EF08EEFFE
:1025100012F00401500E826F96EC0EF0EFEF29F0EE
:10252000C90E64EC0BF0E8CF0BF004012C0E826FA7
:1025300096EC0EF003018451450AD8B4AEEF12F0C8
:1025400003018451440AD8B4B1EF12F0030184515D
:102550004D0AD8B4B4EF12F0C2EF12F00B9EBCEFEC
:1025600012F00B8EBCEF12F0F80E0B1685C3E8FFCD
:10257000070B0B12BCEF12F0C90E0C6E0BC00BF068
:102580004DEC0BF00401310E826F96EC0EF004015D
:102590002C0E826F96EC0EF0C90E64EC0BF0E8CFB7
:1025A0001AF01ABE06D00401450E826F96EC0EF0AA
:1025B00005D00401440E826F96EC0EF004012C0E3F
:1025C000826F96EC0EF01AC0E8FF070BE8CF82F49A
:1025D0000401300E822796EC0EF004012C0E826F5F
:1025E00096EC0EF00780EEEC30F02BC0E8FF003BDD
:1025F00000430043030B77EC30F033C182F4040155
:10260000300E822796EC0EF004012C0E826F96ECB1
:102610000EF0EEEC30F02BC001F1019F019D2CC0BB
:1026200000F1010177EC30F02FC182F40401300E8B
:10263000822796EC0EF030C182F40401300E82271E
:1026400096EC0EF031C182F40401300E822796EC34
:102650000EF032C182F40401300E822796EC0EF0A7
:1026600033C182F40401300E822796EC0EF004018F
:102670002C0E826F96EC0EF0EEEC30F02DC001F1D6
:102680002EC000F1D89001330033D89001330033CD
:10269000010177EC30F02FC182F40401300E822763
:1026A00096EC0EF030C182F40401300E822796ECD5
:1026B0000EF031C182F40401300E822796EC0EF048
:1026C00032C182F40401300E822796EC0EF033C141
:1026D00082F40401300E822796EC0EF0EFEF29F021
:1026E000FC0E64EC0BF0E8CF0BF003018351520AAF
:1026F000D8B4A7EF13F003018351720AD8B4AAEF3C
:1027000013F003018351500AD8B4ADEF13F0030165
:102710008351700AD8B4B0EF13F003018351550A06
:10272000D8B4B3EF13F003018351750AD8B4B6EFF0
:1027300013F003018351430AD8B4BFEF13F0030130
:102740008351630AD8B4C2EF13F0CBEF13F00B90B0
:10275000C5EF13F00B80C5EF13F00B92C5EF13F02C
:102760000B82C5EF13F00B94C5EF13F00B84C5EF8C
:1027700013F00B96C5EF13F00B86C5EF13F00B9813
:10278000C5EF13F00B88C5EF13F0FC0E0C6E0BC0F9
:102790000BF04DEC0BF00401590E826F96EC0EF02D
:1027A0001190119211941198FC0E64EC0BF0E8CF8B
:1027B0000BF00BA011800BA211820BA411840BA8AB
:1027C000118811A0EBEF13F00401520E826F96EC0A
:1027D0000EF0F0EF13F00401720E826F96EC0EF023
:1027E00011A8FAEF13F00401430E826F96EC0EF07D
:1027F000FFEF13F00401630E826F96EC0EF011A24E
:1028000009EF14F00401500E826F96EC0EF00EEFFB
:1028100014F00401700E826F96EC0EF011A418EF04
:1028200014F00401550E826F96EC0EF01DEF14F0BB
:102830000401750E826F96EC0EF0EFEF29F00401A3
:102840006D0E826F96EC0EF003018351300AD8B4FE
:1028500077EF14F003018351310AD8B48AEF14F0F2
:1028600003018351320AD8B49DEF14F0F1EF29F03F
:1028700004014D0E826F96EC0EF02FEC31F084C304
:1028800031F185C332F186C333F10101296B3CEC90
:1028900031F0B3EC30F003018351300AD8B45FEF6C
:1028A00014F003018351310AD8B467EF14F0030127
:1028B0008351320AD8B46FEF14F0F1EF29F0FD0E16
:1028C0000C6E00C10BF04DEC0BF077EF14F0FE0E28
:1028D0000C6E00C10BF04DEC0BF08AEF14F0FF0E04
:1028E0000C6E00C10BF04DEC0BF09DEF14F00401E9
:1028F000300E826F96EC0EF004012C0E826F96EC77
:102900000EF0EEEC30F0FD0E64EC0BF0E8CF00F1D1
:10291000AEEF14F00401310E826F96EC0EF004015C
:102920002C0E826F96EC0EF0EEEC30F0FE0E64ECA6
:102930000BF0E8CF00F1AEEF14F00401320E826F1D
:1029400096EC0EF0EEEC30F004012C0E826F96EC5B
:102950000EF0FF0E64EC0BF0E8CF00F177EC30F0F6
:1029600031C182F40401300E822796EC0EF032C1A0
:1029700082F40401300E822796EC0EF033C182F40B
:102980000401300E822796EC0EF0EFEF29F00301E0
:102990008351300AD8B41BEF1AF003018351310A76
:1029A000D8B448EF1BF003018351320AD8B4B6EF14
:1029B0001BF003018351330AD8B4C6EF1BF00301A7
:1029C0008351340AD8B421EF1CF003018351350A36
:1029D000D8B4F5EF1DF003018351360AD8B423EFC4
:1029E0001EF003018351370AD8B4F3EF17F0030147
:1029F0008351380AD8B491EF18F003018351440A87
:102A0000D8B41FEF16F003018351640AD8B43FEF26
:102A100016F003018351460AD8B4FAEF1CF0030103
:102A200083514D0AD8B46CEF16F0030183516D0A3F
:102A3000D8B486EF16F0030183515A0AD8B4C2EF16
:102A40001AF003018351490AD8B423EF1FF00301A0
:102A50008351500AD8B455EF1EF003018351540A34
:102A6000D8B4CEEF1EF003018351630AD8B4A6EFA9
:102A700016F003018351430AD8B49EEF17F0030107
:102A80008351730AD8B4A4EF16F003018351610A8D
:102A9000D8B46CEF15F003018351650AD8B46BEF1D
:102AA0001AF003018351450AD8B479EF1AF00301F3
:102AB0008351620AD8B487EF1AF003018351420AA6
:102AC000D8B495EF1AF003018351760AD8B4A3EF76
:102AD0001AF0D8A4F1EF29F004014C0E826F96ECA5
:102AE0000EF00401610E826F96EC0EF037EC32F0BE
:102AF00004012C0E826F96EC0EF0EEEC30F0AFC5B8
:102B000000F1010177EC30F031C182F40401300EA4
:102B1000822796EC0EF032C182F40401300E822737
:102B200096EC0EF033C182F40401300E822796EC4D
:102B30000EF004012C0E826F96EC0EF0EEEC30F0ED
:102B4000B0C500F1010177EC30F031C182F404012D
:102B5000300E822796EC0EF032C182F40401300E62
:102B6000822796EC0EF033C182F40401300E8227E6
:102B700096EC0EF004012C0E826F96EC0EF0EEEC4B
:102B800030F0B1C500F1010177EC30F031C182F4D1
:102B90000401300E822796EC0EF032C182F404015B
:102BA000300E822796EC0EF033C182F40401300E11
:102BB000822796EC0EF004012C0E826F96EC0EF03C
:102BC000EEEC30F0B2C500F1010177EC30F031C12C
:102BD00082F40401300E822796EC0EF032C182F4AA
:102BE0000401300E822796EC0EF033C182F404010A
:102BF000300E822796EC0EF004012C0E826F96ECBC
:102C00000EF0EEEC30F0B6C500F1010177EC30F0DB
:102C100031C182F40401300E822796EC0EF032C1ED
:102C200082F40401300E822796EC0EF033C182F458
:102C30000401300E822796EC0EF051EF1EF00301D6
:102C40008451300AD8B42BEF16F003018451310AB5
:102C5000D8B42FEF16F01592159630EF16F01582B6
:102C6000C70E64EC0BF0E8CF00F10101008115A262
:102C70000091C70E0C6E00C10BF04DEC0BF0C70EAF
:102C800064EC0BF0E8CF00F1010100B14BEF16F05E
:102C900015924CEF16F0158204014C0E826F96ECE3
:102CA0000EF00401640E826F96EC0EF004012C0EFF
:102CB000826F96EC0EF015B265EF16F00401300E3F
:102CC000826F96EC0EF06AEF16F00401310E826FFF
:102CD00096EC0EF0EFEF29F02FEC31F084C333F1D6
:102CE0003CEC31F0B3EC30F0200E0C6E00C10BF078
:102CF0004DEC0BF000C12FF505012F51000A06E045
:102D000005012F51010A02E0D1EC32F004014C0E12
:102D1000826F96EC0EF004014D0E826F96EC0EF071
:102D200004012C0E826F96EC0EF0EEEC30F02FC505
:102D300000F177EC30F033C182F40401300E8227C9
:102D400096EC0EF051EF1EF0B3EF38F004014C0E8C
:102D5000826F96EC0EF00401630E826F96EC0EF01B
:102D60008FEC31F004012C0E826F96EC0EF0BBEC70
:102D700016F051EF1EF0EEEC30F0B5C500F1010198
:102D8000003B0F0E001777EC30F033C182F40401E2
:102D9000300E822796EC0EF0B5C500F101010F0E42
:102DA0000101001777EC30F033C182F40401300EDA
:102DB000822796EC0EF004012D0E826F96EC0EF039
:102DC000B4C500F10101003B0F0E001777EC30F0A5
:102DD00033C182F40401300E822796EC0EF0B4C5A4
:102DE00000F101010F0E0101001777EC30F033C143
:102DF00082F40401300E822796EC0EF004012D0EB1
:102E0000826F96EC0EF0B3C500F10101003B0F0E8E
:102E1000001777EC30F033C182F40401300E8227C2
:102E200096EC0EF0B3C500F101010F0E0101001781
:102E300077EC30F033C182F40401300E822796EC37
:102E40000EF00401200E826F96EC0EF0B2C500F178
:102E50000F0E0101001777EC30F033C182F404014A
:102E6000300E822796EC0EF00401200E826F96EC55
:102E70000EF0B1C500F101010101003B0F0E00177A
:102E800077EC30F033C182F40401300E822796ECE7
:102E90000EF0B1C500F101010F0E0101001777EC32
:102EA00030F033C182F40401300E822796EC0EF02C
:102EB00004013A0E826F96EC0EF0B0C500F10101EC
:102EC000003B0F0E001777EC30F033C182F40401A1
:102ED000300E822796EC0EF0B0C500F101010F0E06
:102EE0000101001777EC30F033C182F40401300E99
:102EF000822796EC0EF004013A0E826F96EC0EF0EB
:102F0000AFC500F10101003B0F0E001777EC30F068
:102F100033C182F40401300E822796EC0EF0AFC567
:102F200000F101010F0E001777EC30F033C182F48D
:102F30000401300E822796EC0EF0120084C3E8FFE5
:102F40000F0BE83AE8CFB5F585C3E8FF0F0B050195
:102F5000B51387C3E8FF0F0BE83AE8CFB4F588C391
:102F6000E8FF0F0B0501B4138AC3E8FF0F0BE83A23
:102F7000E8CFB3F58BC3E8FF0F0B0501B3138DC387
:102F8000E8FF0F0BE8CFB2F58FC3E8FF0F0BE83A6D
:102F9000E8CFB1F590C3E8FF0F0B0501B11392C361
:102FA000E8FF0F0BE83AE8CFB0F593C3E8FF0F0B4B
:102FB0000501B01395C3E8FF0F0BE83AE8CFAFF572
:102FC00096C3E8FF0F0B0501AF13EAEC31F00401E3
:102FD0004C0E826F96EC0EF00401430E826F96EC5D
:102FE0000EF0B0EF16F0078404014C0E826F96ECE1
:102FF0000EF00401370E826F96EC0EF004012C0ED9
:10300000826F96EC0EF005012E51130A06E00501C1
:103010002E51170A0DE08EEF18F00101000E006F1F
:10302000000E016F100E026F000E036F21EF18F0FB
:103030000101000E006F000E016F000E026F010E05
:10304000036F77EC30F02AC182F40401300E82273E
:1030500096EC0EF02BC182F40401300E822796EC20
:103060000EF02CC182F40401300E822796EC0EF093
:103070002DC182F40401300E822796EC0EF02EC191
:1030800082F40401300E822796EC0EF02FC182F4F8
:103090000401300E822796EC0EF030C182F4040158
:1030A000300E822796EC0EF031C182F40401300E0E
:1030B000822796EC0EF032C182F40401300E822792
:1030C00096EC0EF033C182F40401300E822796ECA8
:1030D0000EF004012C0E826F96EC0EF00101100E22
:1030E000006F000E016F000E026F000E036F77EC91
:1030F00030F031C182F40401300E822796EC0EF0DC
:1031000032C182F40401300E822796EC0EF033C1F6
:1031100082F40401300E822796EC0EF0079451EFF2
:103120001EF00501216B226B236B246B04014C0EF6
:10313000826F96EC0EF00401380E826F96EC0EF062
:1031400004012C0E826F96EC0EF00101100E006F40
:10315000000E016F000E026F000E036F77EC30F06F
:103160002AC182F40401300E822796EC0EF02BC1A6
:1031700082F40401300E822796EC0EF02CC182F40A
:103180000401300E822796EC0EF02DC182F404016A
:10319000300E822796EC0EF02EC182F40401300E20
:1031A000822796EC0EF02FC182F40401300E8227A4
:1031B00096EC0EF030C182F40401300E822796ECBA
:1031C0000EF031C182F40401300E822796EC0EF02D
:1031D00032C182F40401300E822796EC0EF033C126
:1031E00082F40401300E822796EC0EF004012C0EBE
:1031F000826F96EC0EF025C500F126C501F127C5BA
:1032000002F128C503F10101100E046F000E056FD5
:10321000000E066F000E076F0AEC30F000C133F5A8
:1032200001C134F502C135F503C136F577EC30F054
:103230002AC182F40401300E822796EC0EF02BC1D5
:1032400082F40401300E822796EC0EF02CC182F439
:103250000401300E822796EC0EF02DC182F4040199
:10326000300E822796EC0EF02EC182F40401300E4F
:10327000822796EC0EF02FC182F40401300E8227D3
:1032800096EC0EF030C182F40401300E822796ECE9
:103290000EF031C182F40401300E822796EC0EF05C
:1032A00032C182F40401300E822796EC0EF033C155
:1032B00082F40401300E822796EC0EF0A0EC0EF0A2
:1032C000050133676BEF19F034676BEF19F0356761
:1032D0006BEF19F0366702D00AEF1AF0129E129CBB
:1032E00021C500F122C501F123C502F124C503F176
:1032F000899A400EC76E200EC66E9E96C69E0B0E15
:10330000C96EFF0E9EB602D0E82EFCD79E96C69ED2
:1033100002C1C9FFFF0E9EB602D0E82EFCD79E96D2
:10332000C69E01C1C9FFFF0E9EB602D0E82EFCD793
:103330009E96C69E00C1C9FFFF0E9EB602D0E82E23
:10334000FCD79E96C69EC952FF0E9EB602D0E82EAE
:10335000FCD70501100E326F040114EE00F080510D
:103360007F0BE1269E96C69EC952FF0E9EB602D0E6
:10337000E82EFCD7C9CFE7FF0401802B0501322FCF
:10338000ACEF19F0898A33C500F134C501F135C5B8
:1033900002F136C503F10101010E046F000E056F45
:1033A000000E066F000E076FD9EC2FF000C133F549
:1033B00001C134F502C135F503C136F505013367A6
:1033C000E9EF19F03467E9EF19F03567E9EF19F023
:1033D000366702D00AEF1AF021C500F122C501F1CB
:1033E00023C502F124C503F10101100E046F000E84
:1033F000056F000E066F000E076FDEEC2FF000C1A8
:1034000021F501C122F502C123F503C124F5128E75
:10341000F1EF29F00401450E826F96EC0EF00401E5
:103420004F0E826F96EC0EF00401460E826F96EC02
:103430000EF051EF1EF007840DEC38F0EEEC30F09A
:103440002DC500F177EC30F004014C0E826F96EC44
:103450000EF00401300E826F96EC0EF004012C0E7B
:10346000826F96EC0EF031C182F40401300E822797
:1034700096EC0EF032C182F40401300E822796ECF5
:103480000EF033C182F40401300E822796EC0EF068
:1034900004012C0E826F96EC0EF0EEEC30F02EC58F
:1034A00000F177EC30F031C182F40401300E822754
:1034B00096EC0EF032C182F40401300E822796ECB5
:1034C0000EF033C182F40401300E822796EC0EF028
:1034D000079451EF1EF004014C0E826F96EC0EF033
:1034E0000401650E826F96EC0EF0ADEC33F051EFF7
:1034F0001EF004014C0E826F96EC0EF00401450E96
:10350000826F96EC0EF0C4EC33F051EF1EF0040124
:103510004C0E826F96EC0EF00401620E826F96ECF8
:103520000EF0F2EC33F051EF1EF004014C0E826FFE
:1035300096EC0EF00401420E826F96EC0EF0DBEC7E
:1035400033F051EF1EF004014C0E826F96EC0EF03A
:103550000401760E826F96EC0EF004012C0E826F41
:1035600096EC0EF010A807D00401310E826F96EC95
:103570000EF051EF1EF00401300E826F96EC0EF04B
:1035800051EF1EF004014C0E826F96EC0EF0040118
:103590005A0E826F96EC0EF004012C0E826F96ECA0
:1035A0000EF00DEC38F0EEEC30F005012E51130A60
:1035B00006E005012E51170A0DE0F3EF1AF00101A4
:1035C000000E006F000E016F100E026F000E036FF1
:1035D000F3EF1AF00101000E006F000E016F000EF4
:1035E000026F010E036F0101100E046F000E056FD4
:1035F000000E066F000E076F0AEC30F077EC30F02B
:103600002AC182F40401300E822796EC0EF02BC101
:1036100082F40401300E822796EC0EF02CC182F465
:103620000401300E822796EC0EF02DC182F40401C5
:10363000300E822796EC0EF02EC182F40401300E7B
:10364000822796EC0EF02FC182F40401300E8227FF
:1036500096EC0EF030C182F40401300E822796EC15
:103660000EF031C182F40401300E822796EC0EF088
:1036700032C182F40401300E822796EC0EF033C181
:1036800082F40401300E822796EC0EF051EF1EF00A
:10369000078404014C0E826F96EC0EF00401310E8B
:1036A000826F96EC0EF004012C0E826F96EC0EF0F9
:1036B00025C500F126C501F127C502F128C503F192
:1036C0000101100E046F000E056F000E066F000E54
:1036D000076F0AEC30F077EC30F02AC182F4040175
:1036E000300E822796EC0EF02BC182F40401300ECE
:1036F000822796EC0EF02CC182F40401300E822752
:1037000096EC0EF02DC182F40401300E822796EC67
:103710000EF02EC182F40401300E822796EC0EF0DA
:103720002FC182F40401300E822796EC0EF030C1D6
:1037300082F40401300E822796EC0EF031C182F43F
:103740000401300E822796EC0EF032C182F404019F
:10375000300E822796EC0EF033C182F40401300E55
:10376000822796EC0EF0079451EF1EF007840401B7
:103770004C0E826F96EC0EF00401320E826F96ECC6
:103780000EF0E1EC35F0079451EF1EF0078437B0EE
:10379000CCEF1BF0DFEF1BF0010E166E04014C0E98
:1037A000826F96EC0EF00401330E826F96EC0EF0F1
:1037B0003EEC36F0000E166E079453EF1BF0020E2F
:1037C000166E3EEC36F08B800501010E306F3C0E1C
:1037D000316F01015E6B5F6B606B616B626B636B82
:1037E000646B656B666B676B686B696B536B546B73
:1037F000CF6ACE6A0F9A0F9C0F9E030E166E0401BD
:103800004C0E826F96EC0EF00401330E826F96EC34
:103810000EF004012C0E826F96EC0EF004012D0EBA
:10382000826F96EC0EF00401310E826F96EC0EF072
:10383000EFEF29F03EEC36F0000E166E8B90F1EFB4
:1038400029F0078404014C0E826F96EC0EF00401FF
:10385000340E826F96EC0EF004012C0E826F96EC03
:103860000EF02FEC31F084C32AF185C32BF186C30F
:103870002CF187C32DF188C32EF189C32FF18AC3A0
:1038800030F18BC331F18CC332F18DC333F10101BF
:10389000296B3CEC31F0B3EC30F0100E046F000EED
:1038A000056F000E066F000E076FEAEC2FF000C1E7
:1038B00021F501C122F502C123F503C124F5C0ECB5
:1038C00037F038C5AFF539C5B0F53AC5B1F53BC5E8
:1038D000B2F53CC5B3F53DC5B4F53EC5B5F5BBEC99
:1038E00016F004012C0E826F96EC0EF03FC500F12D
:1038F00040C501F141C502F142C503F10101000ECD
:10390000046F000E056F010E066F000E076F0AECC4
:1039100030F077EC30F0296790EF1CF095EF1CF059
:1039200004012D0E826F96EC0EF030C182F404017A
:10393000300E822796EC0EF031C182F40401300E75
:10394000822796EC0EF004012E0E826F96EC0EF09C
:1039500032C182F40401300E822796EC0EF033C19E
:1039600082F40401300E822796EC0EF004012C0E36
:10397000826F96EC0EF0EEEC30F043C500F144C5DA
:1039800001F11BEC2BF004012C0E826F96EC0EF073
:10399000EEEC30F045C500F177EC30F031C182F447
:1039A0000401300E822796EC0EF032C182F404013D
:1039B000300E822796EC0EF033C182F40401300EF3
:1039C000822796EC0EF004012C0E826F96EC0EF01E
:1039D00037C5E8FFE8B806D00401300E826F96ECD8
:1039E0000EF005D00401310E826F96EC0EF00794B4
:1039F00051EF1EF02FEC31F085C32AF186C32BF175
:103A000087C32CF188C32DF189C32EF18AC32FF10E
:103A10008BC330F18CC331F18DC332F18EC333F1DE
:103A20000101296B3CEC31F0B3EC30F00101010EE7
:103A3000046F000E056F000E066F000E076FD9ECC5
:103A40002FF0100E046F000E056F000E066F000EB3
:103A5000076FEAEC2FF000C129F501C12AF502C178
:103A60002BF503C12CF568EC35F004014C0E826F88
:103A700096EC0EF00401460E826F96EC0EF00401F7
:103A80002C0E826F96EC0EF025C500F126C501F1D3
:103A900027C502F128C503F10101100E046F000EC5
:103AA000056F000E066F000E076F0AEC30F077EC22
:103AB00030F02AC182F40401300E822796EC0EF019
:103AC0002BC182F40401300E822796EC0EF02CC13B
:103AD00082F40401300E822796EC0EF02DC182F4A0
:103AE0000401300E822796EC0EF02EC182F4040100
:103AF000300E822796EC0EF02FC182F40401300EB6
:103B0000822796EC0EF030C182F40401300E822739
:103B100096EC0EF031C182F40401300E822796EC4F
:103B20000EF032C182F40401300E822796EC0EF0C2
:103B300033C182F40401300E822796EC0EF051EF6F
:103B40001EF037B0A6EF1DF0020E166E3EEC36F0FA
:103B500000011650020AD8B4C4EF1DF005012F5120
:103B6000010AD8B4BAEF1DF015B2BFEF1DF081BA4B
:103B7000BFEF1DF0000E166E1584F1EF29F0050E53
:103B8000166E1584B3EF38F08B8001015E6B5F6BAE
:103B9000606B616B626B636B646B656B666B676BB1
:103BA000686B696B536B546BCF6ACE6A0F9A0F9C2C
:103BB0000F9E030E166EF1EF29F03EEC36F0050174
:103BC0002F51010AD8B4EBEF1DF015B2F0EF1DF044
:103BD00081BAF0EF1DF0000E166E1584F1EF29F09A
:103BE000050E166E1584B3EF38F004014C0E826F8B
:103BF00096EC0EF00401350E826F96EC0EF0040187
:103C00002C0E826F96EC0EF0EEEC30F00784B9C506
:103C100000F1079477EC30F031C182F40401300EEA
:103C2000822796EC0EF032C182F40401300E822716
:103C300096EC0EF033C182F40401300E822796EC2C
:103C40000EF051EF1EF001EC36F0EEEC30F037C51F
:103C500000F177EC30F004014C0E826F96EC0EF020
:103C60000401360E826F96EC0EF004012C0E826F6A
:103C700096EC0EF031C182F40401300E822796ECEE
:103C80000EF032C182F40401300E822796EC0EF061
:103C900033C182F40401300E822796EC0EF051EF0E
:103CA0001EF0A0EC0EF0F1EF29F004014C0E826F33
:103CB00096EC0EF00401500E826F96EC0EF00401AB
:103CC0002C0E826F96EC0EF085C32AF186C32BF181
:103CD00087C32CF188C32DF189C32EF18AC32FF13C
:103CE0008BC330F18CC331F18DC332F18EC333F10C
:103CF00001013CEC31F0B3EC30F003018451530A84
:103D00000DE0030184514D0A38E00401780E826F02
:103D100096EC0EF0A0EC0EF0F1EF29F00401530E3A
:103D2000826F96EC0EF0250E0C6E00C10BF04DEC80
:103D30000BF0260E0C6E01C10BF04DEC0BF0270EB4
:103D40000C6E02C10BF04DEC0BF0280E0C6E03C193
:103D50000BF04DEC0BF000C157F501C158F502C155
:103D600059F503C15AF500C15BF501C15CF502C10B
:103D70005DF503C15EF532EF1FF004014D0E826F59
:103D800096EC0EF0290E0C6E00C10BF04DEC0BF012
:103D900000C15FF500C160F532EF1FF004014C0E69
:103DA000826F96EC0EF00401540E826F96EC0EF0CA
:103DB00004012C0E826F96EC0EF084C32AF185C3A9
:103DC0002BF186C32CF187C32DF188C32EF189C353
:103DD0002FF18AC330F18BC331F18DC332F18EC321
:103DE00033F101013CEC31F0B3EC30F00101000E95
:103DF000046F000E056F010E066F000E076FEAECF0
:103E00002FF0210E0C6E00C10BF04DEC0BF0220ECA
:103E10000C6E01C10BF04DEC0BF0230E0C6E02C1C9
:103E20000BF04DEC0BF0240E0C6E03C10BF04DECBF
:103E30000BF000C161F501C162F502C163F503C178
:103E400064F532EF1FF004014C0E826F96EC0EF019
:103E50000401490E826F96EC0EF004012C0E826F65
:103E600096EC0EF0250E64EC0BF0E8CF00F1260E78
:103E700064EC0BF0E8CF01F1270E64EC0BF0E8CF17
:103E800002F1280E64EC0BF0E8CF03F177EC30F090
:103E90003AEC2EF00401730E826F96EC0EF00401E2
:103EA0002C0E826F96EC0EF0EEEC30F0290E64ECE6
:103EB0000BF0E8CF00F177EC30F03AEC2EF0040193
:103EC0006D0E826F96EC0EF004012C0E826F96EC54
:103ED0000EF05BC500F15CC501F15DC502F15EC588
:103EE00003F177EC30F03AEC2EF00401730E826FA0
:103EF00096EC0EF004012C0E826F96EC0EF0EEECB8
:103F000030F060C500F177EC30F03AEC2EF00401AF
:103F10006D0E826F96EC0EF004012C0E826F96EC03
:103F20000EF061C500F162C501F163C502F164C51F
:103F300003F10CEC2AF004012C0E826F96EC0EF0CB
:103F4000A0EC0EF0F1EF29F083C32AF184C32BF12A
:103F500085C32CF186C32DF187C32EF188C32FF1C1
:103F600089C330F18AC331F18BC332F18CC333F191
:103F700001013CEC31F0B3EC30F0160E0C6E00C1D8
:103F80000BF04DEC0BF0170E0C6E01C10BF04DEC6D
:103F90000BF0180E0C6E02C10BF04DEC0BF0190E6D
:103FA0000C6E03C10BF04DEC0BF000C18EF101C1A2
:103FB0008FF102C190F103C191F100C192F101C1F1
:103FC00093F102C194F103C195F186EF20F083C310
:103FD0002AF184C32BF185C32CF186C32DF187C34D
:103FE0002EF188C32FF189C330F18AC331F18BC31D
:103FF00032F18CC333F101013CEC31F0B3EC30F021
:1040000000C18EF101C18FF102C190F103C191F1A4
:1040100000C192F101C193F102C194F103C195F184
:1040200086EF20F083C32AF184C32BF185C32CF1E2
:1040300086C32DF187C32EF188C32FF189C330F1D8
:104040008AC331F18CC332F18DC333F101013CECF1
:1040500031F0B3EC30F00101000E046F000E056F7B
:10406000010E066F000E076FEAEC2FF01A0E0C6EB1
:1040700000C10BF04DEC0BF01B0E0C6E01C10BF0F0
:104080004DEC0BF01C0E0C6E02C10BF04DEC0BF066
:104090001D0E0C6E03C10BF04DEC0BF000C196F140
:1040A00001C197F102C198F103C199F186EF20F0A7
:1040B00083C32AF184C32BF185C32CF186C32DF170
:1040C00087C32EF188C32FF189C330F18AC331F140
:1040D0008CC332F18DC333F101013CEC31F0B3EC10
:1040E00030F00101000E046F000E056F010E066F27
:1040F000000E076FEAEC2FF000C196F101C197F1B5
:1041000002C198F103C199F186EF20F0160E64EC1C
:104110000BF0E8CF00F1170E64EC0BF0E8CF01F1E3
:10412000180E64EC0BF0E8CF02F1190E64EC0BF002
:10413000E8CF03F177EC30F03AEC2EF00401730E87
:10414000826F96EC0EF004012C0E826F96EC0EF04E
:104150008EC100F18FC101F190C102F191C103F153
:1041600077EC30F03AEC2EF00401730E826F96EC8F
:104170000EF004012C0E826F96EC0EF01A0E64EC19
:104180000BF0E8CF00F11B0E64EC0BF0E8CF01F16F
:104190001C0E64EC0BF0E8CF02F11D0E64EC0BF08A
:1041A000E8CF03F10CEC2AF004012C0E826F96ECA0
:1041B0000EF096C100F197C101F198C102F199C1C9
:1041C00003F10CEC2AF0A0EC0EF0F1EF29F0040161
:1041D000690E826F96EC0EF004012C0E826F96EC45
:1041E0000EF00101040E006F000E016F000E026F51
:1041F000000E036F77EC30F02CC182F40401300E16
:10420000822796EC0EF02DC182F40401300E822735
:1042100096EC0EF02EC182F40401300E822796EC4B
:104220000EF02FC182F40401300E822796EC0EF0BE
:1042300030C182F40401300E822796EC0EF031C1B9
:1042400082F40401300E822796EC0EF032C182F423
:104250000401300E822796EC0EF033C182F4040183
:10426000300E822796EC0EF004012C0E826F96EC35
:104270000EF00101060E006F000E016F000E026FBE
:10428000000E036F77EC30F02CC182F40401300E85
:10429000822796EC0EF02DC182F40401300E8227A5
:1042A00096EC0EF02EC182F40401300E822796ECBB
:1042B0000EF02FC182F40401300E822796EC0EF02E
:1042C00030C182F40401300E822796EC0EF031C129
:1042D00082F40401300E822796EC0EF032C182F493
:1042E0000401300E822796EC0EF033C182F40401F3
:1042F000300E822796EC0EF004012C0E826F96ECA5
:104300000EF001014B0E006F000E016F000E026FE8
:10431000000E036F77EC30F02CC182F40401300EF4
:10432000822796EC0EF02DC182F40401300E822714
:1043300096EC0EF02EC182F40401300E822796EC2A
:104340000EF02FC182F40401300E822796EC0EF09D
:1043500030C182F40401300E822796EC0EF031C198
:1043600082F40401300E822796EC0EF032C182F402
:104370000401300E822796EC0EF033C182F4040162
:10438000300E822796EC0EF004012C0E826F96EC14
:104390000EF0200EF86EF76AF66A04010900F5CFF8
:1043A00082F496EC0EF00900F5CF82F496EC0EF054
:1043B0000900F5CF82F496EC0EF00900F5CF82F4F7
:1043C00096EC0EF00900F5CF82F496EC0EF00900A1
:1043D000F5CF82F496EC0EF00900F5CF82F496EC5E
:1043E0000EF00900F5CF82F496EC0EF0A0EC0EF082
:1043F000F1EF29F08351630AD8A4EFEF29F084513B
:10440000610AD8A4EFEF29F085516C0AD8A4EFEF28
:1044100029F08651410A3FE08651440A1BE086514B
:10442000420AD8B45EEF22F08651350AD8B47BEF49
:104430002BF08651360AD8B4D0EF2BF08651370ACC
:10444000D8B439EF2CF08651380AD8B497EF2CF055
:10445000EFEF29F00798079A04017A0E826F96EC25
:104460000EF00401780E826F96EC0EF00401640EDB
:10447000826F96EC0EF00401550E826F96EC0EF0F2
:1044800047EF22F004014C0E826F96EC0EF0A0EC88
:104490000EF0F1EF29F00788079A04017A0E826F77
:1044A00096EC0EF00401410E826F96EC0EF00401C2
:1044B000610E826F96EC0EF03BEF22F00798078AB0
:1044C00004017A0E826F96EC0EF00401420E826FA8
:1044D00096EC0EF00401610E826F96EC0EF03BEF4D
:1044E00022F0010166677CEF22F067677CEF22F023
:1044F00068677CEF22F0696716D001014F6788EF8B
:1045000022F0506788EF22F0516788EF22F052675F
:104510000AD00101000E006F000E016F000E026F45
:10452000000E036F120011B80AD00101620E046F71
:10453000010E056F000E066F000E076F09D0010116
:10454000A70E046F020E056F000E066F000E076FB8
:1045500066C100F167C101F168C102F169C103F1EF
:10456000D9EC2FF003BF25EF23F0119A119C010124
:10457000000E046FA80E056F550E066F020E076F32
:1045800066C100F167C101F168C102F169C103F1BF
:1045900066C18AF167C18BF168C18CF169C18DF187
:1045A000D9EC2FF003BF0BD00101000E8A6FA80ECB
:1045B0008B6F550E8C6F020E8D6F118A119C0E0E33
:1045C00064EC0BF0E8CF18F10F0E64EC0BF0E8CFC1
:1045D00019F1100E64EC0BF0E8CF1AF1110E64EC37
:1045E0000BF0E8CF1BF122EC2FF08AC104F18BC154
:1045F00005F18CC106F18DC107F1D9EC2FF00782CE
:10460000E6EC2EF022EC2FF00792E6EC2EF08AC1B9
:1046100000F18BC101F18CC102F18DC103F1079250
:10462000E6EC2EF0CC0E046FE00E056F870E066FE1
:10463000050E076FD9EC2FF000C118F101C119F177
:1046400002C11AF103C11BF140D013AA2AEF23F0D3
:10465000138E139A119C119A0101800E006F1A0E8D
:10466000016F060E026F000E036F4FC104F150C1BF
:1046700005F151C106F152C107F1D9EC2FF003AF9A
:1046800005D0EEEC30F0118C119A12000E0E64EC95
:104690000BF0E8CF18F10F0E64EC0BF0E8CF19F136
:1046A000100E64EC0BF0E8CF1AF1110E64EC0BF075
:1046B000E8CF1BF14FC100F150C101F151C102F12E
:1046C00052C103F10782E6EC2EF018C100F119C1C6
:1046D00001F11AC102F11BC103F112000784BAC132
:1046E00066F1BBC167F1BCC168F1BDC169F14BC1E5
:1046F0004FF14CC150F14DC151F14EC152F157C172
:1047000059F158C15AF10794010166678FEF23F000
:1047100067678FEF23F068678FEF23F0696716D024
:1047200001014F679BEF23F050679BEF23F0516728
:104730009BEF23F052670AD00101000E006F000EBC
:10474000016F000E026F000E036F120011B80AD045
:104750000101620E046F010E056F000E066F000E60
:10476000076F09D00101A70E046F020E056F000E3E
:10477000066F000E076F66C100F167C101F168C1E5
:1047800002F169C103F1D9EC2FF003BF27EF24F048
:104790000101000E046FA80E056F550E066F020E84
:1047A000076F66C100F167C101F168C102F169C11B
:1047B00003F166C18AF167C18BF168C18CF169C1EF
:1047C0008DF1D9EC2FF003BF09D00101000E8A6FE3
:1047D000A80E8B6F550E8C6F020E8D6F22EC2FF092
:1047E00000C104F101C105F102C106F103C107F1E5
:1047F000000E006FA00E016F980E026F7B0E036F0C
:104800000AEC30F000C118F101C119F102C11AF12E
:1048100003C11BF1000E006FA00E016F980E026F16
:104820007B0E036F8AC104F18BC105F18CC106F1C7
:104830008DC107F10AEC30F018C104F119C105F17E
:104840001AC106F11BC107F1D9EC2FF012000101CA
:10485000A80E006F610E016F000E026F000E036F55
:104860004FC104F150C105F151C106F152C107F128
:10487000D9EC2FF003AF0AD00101A80E006F610E32
:10488000016F000E026F000E036F00D0C80E006FA4
:10489000AF0E016F000E026F000E036F4FC104F1E7
:1048A00050C105F151C106F152C107F1EAEC2FF0F8
:1048B00012000401730E826F96EC0EF004012C0EB0
:1048C000826F96EC0EF0078462C166F163C167F1F6
:1048D00064C168F165C169F14BC14FF14CC150F140
:1048E0004DC151F14EC152F157C159F158C15AF160
:1048F00007947FEC24F0A0EC0EF0F1EF29F066C1F4
:1049000000F167C101F168C102F169C103F1010160
:1049100077EC30F03AEC2EF00401630E826F96ECE7
:104920000EF004012C0E826F96EC0EF04FC100F1D8
:1049300050C101F151C102F152C103F1010177EC03
:1049400030F03AEC2EF00401660E826F96EC0EF019
:1049500004012C0E826F96EC0EF0EEEC30F059C193
:1049600000F15AC101F1010177EC30F03AEC2EF080
:104970000401740E826F96EC0EF012001082040196
:10498000530E826F96EC0EF004012C0E826F96ECA3
:104990000EF083C32AF184C32BF185C32CF186C3A7
:1049A0002DF187C32EF188C32FF189C330F18AC35B
:1049B00031F18BC332F18CC333F101013CEC31F0A6
:1049C000B3EC30F000C166F101C167F102C168F1DA
:1049D00003C169F18EC32AF18FC32BF190C32CF16F
:1049E00091C32DF192C32EF193C32FF194C330F1F3
:1049F00095C331F196C332F197C333F101013CEC19
:104A000031F0B3EC30F000C14FF101C150F102C1FF
:104A100051F103C152F12FEC31F099C32FF19AC338
:104A200030F19BC331F19CC332F19DC333F10101DD
:104A30003CEC31F0B3EC30F000C159F101C15AF156
:104A40007FEC24F004012C0E826F96EC0EF039EF0F
:104A500025F0118E1CA002D01CAE108C1BBE02D003
:104A60001BA4108E03018251520A02E10F8201D071
:104A70000F928251750A02E1108401D01094825184
:104A8000550A02E1108601D010968351310A03E1E4
:104A90001382138402D01392139403018351660A84
:104AA00001E056D00401660E826F96EC0EF0040110
:104AB0002C0E826F96EC0EF06EEC23F077EC30F05B
:104AC0002AC182F40401300E822796EC0EF02BC12D
:104AD00082F40401300E822796EC0EF02CC182F491
:104AE0000401300E822796EC0EF02DC182F40401F1
:104AF000300E822796EC0EF02EC182F40401300EA7
:104B0000822796EC0EF02FC182F40401300E82272A
:104B100096EC0EF030C182F40401300E822796EC40
:104B20000EF031C182F40401300E822796EC0EF0B3
:104B300032C182F40401300E822796EC0EF033C1AC
:104B400082F40401300E822796EC0EF0EFEF29F08C
:104B500011A003D011A401D01084078410B212EF69
:104B600026F010A4F6EF25F0BAC166F1BBC167F1DB
:104B7000BCC168F1BDC169F1BEC16AF1BFC16BF1D1
:104B8000C0C16CF1C1C16DF1C2C16EF1C3C16FF1A1
:104B9000C4C170F1C5C171F1C6C172F1C7C173F171
:104BA000C8C174F1C9C175F1CAC176F1CBC177F141
:104BB000CCC178F1CDC179F1CEC17AF1CFC17BF111
:104BC000D0C17CF1D1C17DF1D2C17EF1D3C17FF1E1
:104BD000D4C180F1D5C181F1D6C182F1D7C183F1B1
:104BE000D8C184F1D9C185F1FEEF25F062C166F12B
:104BF00063C167F164C168F165C169F1BAC186F149
:104C0000BBC187F1BCC188F1BDC189F14BC14FF176
:104C10004CC150F14DC151F14EC152F157C159F142
:104C200058C15AF107940FA034EF26F0010196679E
:104C300021EF26F0976721EF26F0986721EF26F005
:104C4000996725EF26F034EF26F071EC22F096C13B
:104C500004F197C105F198C106F199C107F1D9ECAA
:104C60002FF003BFB5EF29F071EC22F00101000E27
:104C7000046F000E056F010E066F000E076F0AEC41
:104C800030F011A02AD011A228D077EC30F029679B
:104C900001D005D004012D0E826F96EC0EF030C1CC
:104CA00082F40401300E822796EC0EF031C182F4BA
:104CB0000401300E822796EC0EF032C182F404011A
:104CC000300E822796EC0EF033C182F40401300ED0
:104CD000822796EC0EF0A0EC0EF012A8C5D0129828
:104CE0001DC01EF01E3A1E42070E1E1600011E5069
:104CF000000AD8B400EF27F000011E50010AD8B412
:104D00008CEF26F000011E50020AD8B48AEF26F07C
:104D100032EF27F032EF27F0EEEC30F02DC001F14A
:104D20002EC000F1D89001330033D8900133003306
:104D30000101630E046F000E056F000E066F000E7A
:104D4000076F0AEC30F0280E046F000E056F000E9E
:104D5000066F000E076FD9EC2FF000C130F0EEECBB
:104D600030F02BC001F1019F019D2CC000F1010129
:104D7000A40E046F000E056F000E066F000E076F85
:104D80000AEC30F000C12FF000C104F101C105F1BF
:104D900002C106F103C107F1640E006F000E016F3E
:104DA000000E026F000E036FD9EC2FF0050E046F9A
:104DB000000E056F000E066F000E076F0AEC30F054
:104DC00000C104F101C105F102C106F103C107F1FF
:104DD000EEEC30F030C000F1D9EC2FF000C131F032
:104DE00031C0E8FF050F305C03E78A8432EF27F01B
:104DF00031C0E8FF0A0F305C01E68A9432EF27F0F9
:104E000000C124F101C125F102C126F103C127F13E
:104E1000EEEC30F0F4EC30F01D501F0BE8CF00F159
:104E20000101640E046F000E056F000E066F000E88
:104E3000076FEAEC2FF024C104F125C105F126C16A
:104E400006F127C107F1D9EC2FF003BF02D08A94F5
:104E500001D08A8424C100F125C101F126C102F1EB
:104E600027C103F1F1EF29F000C124F101C125F1BF
:104E700002C126F103C127F110AE4DD0109E00C132
:104E800008F101C109F102C10AF103C10BF177EC8C
:104E900030F030C1E2F131C1E3F132C1E4F133C1AC
:104EA000E5F108C100F109C101F10AC102F10BC12C
:104EB00003F101016C0E046F070E056F000E066F03
:104EC000000E076FD9EC2FF003BF04D00101550E7F
:104ED000E66F1CD008C100F109C101F10AC102F15D
:104EE0000BC103F10101A40E046F060E056F000E45
:104EF000066F000E076FD9EC2FF003BF04D001013D
:104F00007F0EE66F03D00101FF0EE66F1F8E11AE1C
:104F1000B5EF29F0119E24C100F125C101F126C190
:104F200002F127C103F111A005D011A203D00FB0E7
:104F3000B5EF29F010A4A4EF27F00401750E826FDD
:104F400096EC0EF0A9EF27F00401720E826F96EC3A
:104F50000EF004012C0E826F96EC0EF077EC30F020
:104F60002967B8EF27F00401200E826FBBEF27F00E
:104F700004012D0E826F96EC0EF030C182F4040114
:104F8000300E822796EC0EF031C182F40401300E0F
:104F9000822796EC0EF004012E0E826F96EC0EF036
:104FA00032C182F40401300E822796EC0EF033C138
:104FB00082F40401300E822796EC0EF004016D0E8F
:104FC000826F96EC0EF004012C0E826F96EC0EF0C0
:104FD0004FC100F150C101F151C102F152C103F1C1
:104FE000010177EC30F03AEC2EF00401480E826FAC
:104FF00096EC0EF004017A0E826F96EC0EF004012E
:105000002C0E826F96EC0EF066C100F167C101F1C3
:1050100068C102F169C103F1010177EC30F03AECAB
:105020002EF00401630E826F96EC0EF004012C0E3C
:10503000826F96EC0EF066C100F167C101F168C1A4
:1050400002F169C103F101010A0E046F000E056F40
:10505000000E066F000E076FEAEC2FF0000E046FD3
:10506000120E056F000E066F000E076F0AEC30F08F
:1050700077EC30F02AC182F40401300E822796ECDE
:105080000EF02BC182F40401300E822796EC0EF054
:105090002CC182F40401300E822796EC0EF02DC153
:1050A00082F40401300E822796EC0EF02EC182F4B9
:1050B0000401300E822796EC0EF02FC182F4040119
:1050C000300E822796EC0EF030C182F40401300ECF
:1050D000822796EC0EF004012E0E826F96EC0EF0F5
:1050E00031C182F40401300E822796EC0EF032C1F9
:1050F00082F40401300E822796EC0EF033C182F464
:105100000401300E822796EC0EF00401730E826FBC
:1051100096EC0EF004012C0E826F96EC0EF0EEEC85
:1051200030F059C100F15AC101F11BEC2BF013A270
:10513000E9EF28F004012C0E826F96EC0EF086C188
:1051400066F187C167F188C168F189C169F171ECC5
:1051500022F00101000E046F000E056F010E066FB4
:10516000000E076F0AEC30F077EC30F02967BEEFE5
:1051700028F00401200E826FC1EF28F004012D0EEB
:10518000826F96EC0EF030C182F40401300E82275B
:1051900096EC0EF031C182F40401300E822796ECB9
:1051A0000EF004012E0E826F96EC0EF032C182F4E6
:1051B0000401300E822796EC0EF033C182F4040114
:1051C000300E822796EC0EF004016D0E826F96EC85
:1051D0000EF003018351460A01E04FD004012C0E6A
:1051E000826F96EC0EF06EEC23F077EC30F02AC173
:1051F00082F40401300E822796EC0EF02BC182F46B
:105200000401300E822796EC0EF02CC182F40401CA
:10521000300E822796EC0EF02DC182F40401300E80
:10522000822796EC0EF02EC182F40401300E822704
:1052300096EC0EF02FC182F40401300E822796EC1A
:105240000EF030C182F40401300E822796EC0EF08D
:1052500031C182F40401300E822796EC0EF032C187
:1052600082F40401300E822796EC0EF033C182F4F2
:105270000401300E822796EC0EF013A464EF29F09F
:1052800004012C0E826F96EC0EF013AC52EF29F055
:105290000401500E826F96EC0EF0139C1398139A33
:1052A00064EF29F013AE5FEF29F00401460E826F20
:1052B00096EC0EF0139E1398139A64EF29F00401F4
:1052C000530E826F96EC0EF037B07BEF29F004019D
:1052D0002C0E826F96EC0EF08BB076EF29F0040165
:1052E000440E826F96EC0EF07BEF29F00401530E12
:1052F000826F96EC0EF00FB281EF29F00FA0B3EFA2
:1053000029F004012C0E826F96EC0EF0200EF86E40
:10531000F76AF66A04010900F5CF82F496EC0EF004
:105320000900F5CF82F496EC0EF00900F5CF82F477
:1053300096EC0EF00900F5CF82F496EC0EF0090021
:10534000F5CF82F496EC0EF00900F5CF82F496ECDE
:105350000EF00900F5CF82F496EC0EF00900F5CFBF
:1053600082F496EC0EF0A0EC0EF00F90109E1298C6
:10537000F1EF29F00401630E826F96EC0EF0040148
:105380002C0E826F96EC0EF0F7EC29F004012C0E37
:10539000826F96EC0EF06AEC2AF004012C0E826FFC
:1053A00096EC0EF0E6EC2AF004012C0E826F96ECDF
:1053B0000EF00101F80E006FCD0E016F660E026F48
:1053C000030E036F0CEC2AF004012C0E826F96EC96
:1053D0000EF0FCEC2AF0A0EC0EF0F1EF29F0A0ECBE
:1053E0000EF00301C26B0790109200EF2DF0D890E1
:1053F0000E0E64EC0BF0E8CF00F10F0E64EC0BF036
:10540000E8CF01F1100E64EC0BF0E8CF02F1110EC1
:1054100064EC0BF0E8CF03F10101000E046F000E05
:10542000056F010E066F000E076F0AEC30F077EC87
:1054300030F02AC182F40401300E822796EC0EF07F
:105440002BC182F40401300E822796EC0EF02CC1A1
:1054500082F40401300E822796EC0EF02DC182F406
:105460000401300E822796EC0EF02EC182F4040166
:10547000300E822796EC0EF02FC182F40401300E1C
:10548000822796EC0EF030C182F40401300E8227A0
:1054900096EC0EF031C182F40401300E822796ECB6
:1054A0000EF004012E0E826F96EC0EF032C182F4E3
:1054B0000401300E822796EC0EF033C182F4040111
:1054C000300E822796EC0EF004016D0E826F96EC82
:1054D0000EF01200120E64EC0BF0E8CF00F1130E88
:1054E00064EC0BF0E8CF01F1140E64EC0BF0E8CFA4
:1054F00002F1150E64EC0BF0E8CF03F101010A0E86
:10550000046F000E056F000E066F000E076FEAECC9
:105510002FF0000E046F120E056F000E066F000EC6
:10552000076F0AEC30F077EC30F02AC182F4040106
:10553000300E822796EC0EF02BC182F40401300E5F
:10554000822796EC0EF02CC182F40401300E8227E3
:1055500096EC0EF02DC182F40401300E822796ECF9
:105560000EF02EC182F40401300E822796EC0EF06C
:105570002FC182F40401300E822796EC0EF030C168
:1055800082F40401300E822796EC0EF004012E0EF8
:10559000826F96EC0EF031C182F40401300E822746
:1055A00096EC0EF032C182F40401300E822796ECA4
:1055B0000EF033C182F40401300E822796EC0EF017
:1055C0000401730E826F96EC0EF012000A0E64EC6A
:1055D0000BF0E8CF00F10B0E64EC0BF0E8CF01F11B
:1055E0000C0E64EC0BF0E8CF02F10D0E64EC0BF046
:1055F000E8CF03F11BEF2BF0060E64EC0BF0E8CFC5
:1056000000F1070E64EC0BF0E8CF01F1080E64EC3A
:105610000BF0E8CF02F1090E64EC0BF0E8CF03F1D8
:105620001BEF2BF00101EEEC30F0078457C100F1C5
:1056300058C101F107940101E80E046F800E056F57
:10564000000E066F000E076FEAEC2FF0000E046FDD
:10565000040E056F000E066F000E076F0AEC30F0A7
:10566000880E046F130E056F000E066F000E076F95
:10567000D9EC2FF00A0E046F000E056F000E066FB6
:10568000000E076F0AEC30F077EC30F0010129676B
:105690004FEF2BF00401200E826F52EF2BF004012C
:1056A0002D0E826F96EC0EF030C182F40401300EA4
:1056B000822796EC0EF031C182F40401300E82276D
:1056C00096EC0EF032C182F40401300E822796EC83
:1056D0000EF004012E0E826F96EC0EF033C182F4B0
:1056E0000401300E822796EC0EF00401430E826F07
:1056F00096EC0EF0120087C32AF188C32BF189C300
:105700002CF18AC32DF18BC32EF18CC32FF18DC3E5
:1057100030F18EC331F190C332F191C333F1010105
:10572000296B3CEC31F0B3EC30F00101000E046F5A
:10573000000E056F010E066F000E076FEAEC2FF0EA
:105740000E0E0C6E00C10BF04DEC0BF00F0E0C6E3C
:1057500001C10BF04DEC0BF0100E0C6E02C10BF002
:105760004DEC0BF0110E0C6E03C10BF04DEC0BF079
:1057700004017A0E826F96EC0EF004012C0E826FFB
:1057800096EC0EF00401350E826F96EC0EF00401DB
:105790002C0E826F96EC0EF0F7EC29F047EF22F01A
:1057A00087C32AF188C32BF189C32CF18AC32DF159
:1057B0008BC32EF18CC32FF18DC330F18EC331F129
:1057C00090C332F191C333F10101296B3CEC31F00C
:1057D000B3EC30F0880E046F130E056F000E066FE9
:1057E000000E076FDEEC2FF0000E046F040E056F45
:1057F000000E066F000E076FEAEC2FF00101E80EB5
:10580000046F800E056F000E066F000E076F0AEC26
:1058100030F00A0E0C6E00C10BF04DEC0BF00B0ECD
:105820000C6E01C10BF04DEC0BF00C0E0C6E02C1B6
:105830000BF04DEC0BF00D0E0C6E03C10BF04DECAC
:105840000BF004017A0E826F96EC0EF004012C0E20
:10585000826F96EC0EF00401360E826F96EC0EF01D
:1058600004012C0E826F96EC0EF0E6EC2AF047EF66
:1058700022F087C32AF188C32BF189C32CF18AC394
:105880002DF18BC32EF18CC32FF18DC330F18FC35B
:1058900031F190C332F191C333F101013CEC31F0AD
:1058A000B3EC30F0000E046F120E056F000E066FA1
:1058B000000E076FEAEC2FF001010A0E046F000ED4
:1058C000056F000E066F000E076F0AEC30F0120E27
:1058D0000C6E00C10BF04DEC0BF0130E0C6E01C101
:1058E0000BF04DEC0BF0140E0C6E02C10BF04DECF6
:1058F0000BF0150E0C6E03C10BF04DEC0BF0040118
:105900007A0E826F96EC0EF004012C0E826F96ECEC
:105910000EF00401370E826F96EC0EF004012C0E8F
:10592000826F96EC0EF06AEC2AF047EF22F087C304
:105930002AF188C32BF189C32CF18AC32DF18BC3C3
:105940002EF18CC32FF18DC330F18EC331F190C392
:1059500032F191C333F10101296B3CEC31F0B3EC2E
:1059600030F0880E046F130E056F000E066F000EE8
:10597000076FDEEC2FF0000E046F040E056F000EB3
:10598000066F000E076FEAEC2FF00101E80E046FBE
:10599000800E056F000E066F000E076F0AEC30F0E8
:1059A000060E0C6E00C10BF04DEC0BF0070E0C6EEA
:1059B00001C10BF04DEC0BF0080E0C6E02C10BF0A8
:1059C0004DEC0BF0090E0C6E03C10BF04DEC0BF01F
:1059D00004017A0E826F96EC0EF004012C0E826F99
:1059E00096EC0EF00401380E826F96EC0EF0040176
:1059F0002C0E826F96EC0EF0FCEC2AF047EF22F0B2
:105A000007A873EF2DF00101800E006F1A0E016FD1
:105A1000060E026F000E036F4BC104F14CC105F17D
:105A20004DC106F14EC107F1D9EC2FF003BFB9EF1C
:105A30002DF034EC2EF04BC100F14CC101F14DC101
:105A400002F14EC103F10782E6EC2EF018C104F119
:105A500019C105F11AC106F11BC107F1F80E006F5B
:105A6000CD0E016F660E026F030E036FD9EC2FF09F
:105A70000E0E0C6E00C10BF04DEC0BF00F0E0C6E09
:105A800001C10BF04DEC0BF0100E0C6E02C10BF0CF
:105A90004DEC0BF0110E0C6E03C10BF04DEC0BF046
:105AA00007840101EEEC30F057C100F158C101F15B
:105AB00007940A0E0C6E00C10BF04DEC0BF00B0EB0
:105AC0000C6E01C10BF04DEC0BF00C0E0C6E02C114
:105AD0000BF04DEC0BF00D0E0C6E03C10BF04DEC0A
:105AE0000BF0B9EF2DF007AAB9EF2DF007840101F3
:105AF000EEEC30F057C100F158C101F10794060EE9
:105B00000C6E00C10BF04DEC0BF0070E0C6E01C1DA
:105B10000BF04DEC0BF0080E0C6E02C10BF04DECCF
:105B20000BF0090E0C6E03C10BF04DEC0BF007846B
:105B300062C100F163C101F164C102F165C103F109
:105B40000794120E0C6E00C10BF04DEC0BF0130E0F
:105B50000C6E01C10BF04DEC0BF0140E0C6E02C17B
:105B60000BF04DEC0BF0150E0C6E03C10BF04DEC71
:105B70000BF00798079A0401805181197F0B0DE003
:105B80009EA8FED714EE00F081517F0BE126E7506E
:105B9000812B0F01AD6EBBEF2DF005012F51000AD7
:105BA000D8B4FCEF2DF081BAE1EF2DF015B2FCEF87
:105BB0002DF005012F51010AD8B4FAEF2DF0F3EFC3
:105BC0002DF005012F51000AD8B4B3EF38F00501CC
:105BD0002F51010AD8B4FAEF2DF000011650050A32
:105BE000D8B4B3EF38F081B8FCEF2DF037EC32F0D9
:105BF00035EC33F04CEC38F0C4EF0DF018C100F187
:105C000019C101F11AC102F11BC103F1000E046FA9
:105C1000000E056F010E066F000E076F0AEC30F0E4
:105C200029A129EF2EF02051D8B429EF2EF018C168
:105C300000F119C101F11AC102F11BC103F1000EFB
:105C4000046F000E056F0A0E066F000E076F0AEC58
:105C500030F01200010104510013055101130651E7
:105C600002130751031312000101186B196B1A6B11
:105C70001B6B12002AC182F40401300E822796ECBD
:105C80000EF02BC182F40401300E822796EC0EF048
:105C90002CC182F40401300E822796EC0EF02DC147
:105CA00082F40401300E822796EC0EF02EC182F4AD
:105CB0000401300E822796EC0EF02FC182F404010D
:105CC000300E822796EC0EF030C182F40401300EC3
:105CD000822796EC0EF031C182F40401300E822747
:105CE00096EC0EF032C182F40401300E822796EC5D
:105CF0000EF033C182F40401300E822796EC0EF0D0
:105D000012002FC182F40401300E822796EC0EF0AF
:105D100030C182F40401300E822796EC0EF031C1BE
:105D200082F40401300E822796EC0EF032C182F428
:105D30000401300E822796EC0EF033C182F4040188
:105D4000300E822796EC0EF01200060E216E060E23
:105D5000226E060E236E212EABEF2EF0222EABEF1D
:105D60002EF0232EABEF2EF08B84020E216E020E4E
:105D7000226E020E236E212EBBEF2EF0222EBBEFE1
:105D80002EF0232EBBEF2EF08B941200FF0E226E0E
:105D900022C023F0030E216E8B84212ECCEF2EF037
:105DA000030E216E232ECCEF2EF08B9422C023F015
:105DB000030E216E212EDAEF2EF0030E216E233E0C
:105DC000DAEF2EF0222EC8EF2EF012000101005360
:105DD00005E1015303E1025301E1002BA9EC2FF08F
:105DE000EEEC30F03951006F3A51016F420E046F02
:105DF0004B0E056F000E066F000E076FEAEC2FF0DA
:105E000000C104F101C105F102C106F103C107F1AE
:105E100018C100F119C101F11AC102F11BC103F14E
:105E200007B217EF2FF0DEEC2FF019EF2FF0D9ECBF
:105E30002FF000C118F101C119F102C11AF103C11B
:105E40001BF11200EEEC30F059C100F15AC101F122
:105E5000060E64EC0BF0E8CF04F1070E64EC0BF0D7
:105E6000E8CF05F1080E64EC0BF0E8CF06F1090E5F
:105E700064EC0BF0E8CF07F1D9EC2FF000C124F16E
:105E800001C125F102C126F103C127F1290E046FDA
:105E9000000E056F000E066F000E076FEAEC2FF084
:105EA000EE0E046F430E056F000E066F000E076FB7
:105EB000DEEC2FF024C104F125C105F126C106F165
:105EC00027C107F1EAEC2FF000C11CF101C11DF15F
:105ED00002C11EF103C11FF1120E64EC0BF0E8CFFA
:105EE00004F1130E64EC0BF0E8CF05F1140E64EC32
:105EF0000BF0E8CF06F1150E64EC0BF0E8CF07F1DC
:105F00000D0E006F000E016F000E026F000E036F8A
:105F1000EAEC2FF0180E046F000E056F000E066FEE
:105F2000000E076F0AEC30F01CC104F11DC105F131
:105F30001EC106F11FC107F1DEEC2FF06A0E046FDF
:105F40002A0E056F000E066F000E076FD9EC2FF0BA
:105F50001200BF0EFA6E200E3A6F396BD8900037E0
:105F6000013702370337D8B0BAEF2FF03A2FAFEF2F
:105F70002FF039073A070353D8B412000331070B47
:105F800080093F6F03390F0B010F396F80EC5FF011
:105F9000406F390580EC5FF0405D405F396B3F3307
:105FA000D8B0392739333FA9CFEF2FF040513927E7
:105FB0001200010113EC31F0D8B0120001010351BD
:105FC0000719346FD6EC30F0D8900751031934AF6D
:105FD000800F12000101346BFAEC30F0D8A010EC05
:105FE00031F0D8B01200E5EC30F0EEEC30F01F0EDE
:105FF000366F26EC31F00B35D8B0D6EC30F0D8A0A7
:106000000335D8B01200362FF9EF2FF034B1FDEC84
:1060100030F012000101346B045105110611071113
:106020000008D8A0FAEC30F0D8A010EC31F0D8B0CD
:106030001200086B096B0A6B0B6B26EC31F01F0E1C
:10604000366F26EC31F007510B5DD8A434EF30F0F9
:1060500006510A5DD8A434EF30F00551095DD8A48B
:1060600034EF30F00451085DD8A047EF30F0045110
:10607000085F0551D8A0053D095F0651D8A0063D2F
:106080000A5F0751D8A0073D0B5FD8900081362FDB
:1060900021EF30F034B1FDEC30F0346BFAEC30F03D
:1060A000D8902AEC31F007510B5DD8A464EF30F0A2
:1060B00006510A5DD8A464EF30F00551095DD8A4FB
:1060C00064EF30F00451085DD8A073EF30F0003F6A
:1060D00073EF30F0013F73EF30F0023F73EF30F0B9
:1060E000032BD8B4120034B1FDEC30F012000101E2
:1060F000346BFAEC30F0D8B012002FEC31F0200EF7
:10610000366F003701370237033711EE33F00A0ECE
:10611000376FE7360A0EE75CD8B0E76EE552372FE7
:1061200089EF30F0362F81EF30F034B12981D890EB
:1061300012002FEC31F0200E366F00370137023796
:10614000033711EE33F00A0E376FE7360A0EE75CBD
:10615000D8B0E76EE552372FA5EF30F0362F9DEF20
:1061600030F0D890120001010A0E346F200E366F05
:1061700011EE29F03451376F0A0ED890E652D8B09C
:10618000E726E732372FBEEF30F003330233013317
:106190000033362FB8EF30F0E750FF0FD8A00335AB
:1061A000D8B0120029B1FDEC30F0120004510027E4
:1061B0000551D8B0053D01270651D8B0063D02274C
:1061C0000751D8B0073D032712000051086F015155
:1061D000096F02510A6F03510B6F12000101006B2E
:1061E000016B026B036B12000101046B056B066B04
:1061F000076B12000335D8A012000351800B001F5B
:10620000011F021F031F003F0DEF31F0013F0DEF93
:1062100031F0023F0DEF31F0032B342B0325120038
:106220000735D8A012000751800B041F051F061F59
:10623000071F043F23EF31F0053F23EF31F0063F06
:1062400023EF31F0072B342B0725120000370137DD
:1062500002370337083709370A370B3712000101B5
:10626000296B2A6B2B6B2C6B2D6B2E6B2F6B306B72
:10627000316B326B336B120001012A510F0B2A6F05
:106280002B510F0B2B6F2C510F0B2C6F2D510F0B14
:106290002D6F2E510F0B2E6F2F510F0B2F6F305173
:1062A0000F0B306F31510F0B316F32510F0B326FBB
:1062B00033510F0B336F120000C124F101C125F1DE
:1062C00002C126F103C127F104C100F105C101F1AA
:1062D00006C102F107C103F124C104F125C105F192
:1062E00026C106F127C107F1120010A806D0899433
:1062F000000EC76E220EC66E05D08984000EC76ED2
:10630000220EC66E050EE82EFED7120010A802D08F
:10631000898401D08994050EE82EFED7120075EC11
:1063200031F09E96C69E000EC96EFF0E9EB602D03C
:10633000E82EFCD79E96C69E000EC96EFF0E9EB636
:1063400002D0E82EFCD7C9CFAFF59E96C69E000EB0
:10635000C96EFF0E9EB602D0E82EFCD7C9CFB0F5AD
:106360009E96C69E000EC96EFF0E9EB602D0E82E07
:10637000FCD7C9CFB1F59E96C69E000EC96EFF0E22
:106380009EB602D0E82EFCD7C9CFB2F59E96C69E27
:10639000000EC96EFF0E9EB602D0E82EFCD7C9CF04
:1063A000B3F59E96C69E000EC96EFF0E9EB602D035
:1063B000E82EFCD7C9CFB4F59E96C69E000EC96ED6
:1063C000FF0E9EB602D0E82EFCD7C9CFB5F586ECFD
:1063D00031F0120075EC31F09E96C69E800EC96EAB
:1063E000FF0E9EB602D0E82EFCD79E96C69EAFC585
:1063F000C9FFFF0E9EB602D0E82EFCD79E96C69E21
:10640000B0C5C9FFFF0E9EB602D0E82EFCD79E96FF
:10641000C69EB1C5C9FFFF0E9EB602D0E82EFCD7BE
:106420009E96C69EB2C5C9FFFF0E9EB602D0E82E4C
:10643000FCD79E96C69EB3C5C9FFFF0E9EB602D07E
:10644000E82EFCD79E96C69EB4C5C9FFFF0E9EB629
:1064500002D0E82EFCD79E96C69EB5C5C9FFFF0E9A
:106460009EB602D0E82EFCD786EC31F0120075EC17
:1064700031F09E96C69E070EC96EFF0E9EB602D0E4
:10648000E82EFCD79E96C69E000EC96EFF0E9EB6E5
:1064900002D0E82EFCD7C9CFAFF59E96C69E000E5F
:1064A000C96EFF0E9EB602D0E82EFCD7C9CFB0F55C
:1064B0009E96C69E000EC96EFF0E9EB602D0E82EB6
:1064C000FCD7C9CFB1F59E96C69E000EC96EFF0ED1
:1064D0009EB602D0E82EFCD7C9CFB2F586EC31F0DB
:1064E00075EC31F09E96C69E25C0C9FFFF0E9EB684
:1064F00002D0E82EFCD79E96C69E000EC96EFF0EF7
:106500009EB602D0E82EFCD7C9CFB6F586EC31F0A6
:10651000120075EC31F09E96C69E870EC96EFF0E76
:106520009EB602D0E82EFCD79E96C69EAFC5C9FF88
:10653000FF0E9EB602D0E82EFCD79E96C69EB0C532
:10654000C9FFFF0E9EB602D0E82EFCD79E96C69ECF
:10655000B1C5C9FFFF0E9EB602D0E82EFCD79E96AD
:10656000C69EB2C5C9FFFF0E9EB602D0E82EFCD76C
:1065700086EC31F075EC31F09E96C69E26C0C9FFC0
:10658000FF0E9EB602D0E82EFCD79E96C69EB6C5DC
:10659000C9FFFF0E9EB602D0E82EFCD786EC31F084
:1065A000120075EC31F09E96C69E870EC96EFF0EE6
:1065B0009EB602D0E82EFCD79E96C69E000EC96EEF
:1065C000FF0E9EB602D0E82EFCD79E96C69E800E89
:1065D000C96EFF0E9EB602D0E82EFCD79E96C69ED0
:1065E000800EC96EFF0E9EB602D0E82EFCD79E9696
:1065F000C69E800EC96EFF0E9EB602D0E82EFCD756
:1066000086EC31F0120075EC31F09E96C69E870E36
:10661000C96EFF0E9EB602D0E82EFCD79E96C69E8F
:10662000000EC96EFF0E9EB602D0E82EFCD79E96D5
:10663000C69E000EC96EFF0E9EB602D0E82EFCD795
:106640009E96C69E800EC96EFF0E9EB602D0E82EA4
:10665000FCD79E96C69E800EC96EFF0E9EB602D0D7
:10666000E82EFCD786EC31F0120010A817D075EC9C
:1066700031F09E96C69E8F0EC96EFF0E9EB602D05A
:10668000E82EFCD79E96C69E000EC96EFF0E9EB6E3
:1066900002D0E82EFCD786EC31F0120037EC32F055
:1066A000120010A82DD075EC31F09E96C69E26C023
:1066B000C9FFFF0E9EB602D0E82EFCD79E96C69E5E
:1066C000450EC96EFF0E9EB602D0E82EFCD786ECB2
:1066D00031F075EC31F09E96C69E8F0EC96EFF0E9E
:1066E0009EB602D0E82EFCD79E96C69E000EC96EBE
:1066F000FF0E9EB602D0E82EFCD786EC31F01200D9
:1067000075EC31F09E96C69E26C0C9FFFF0E9EB660
:1067100002D0E82EFCD79E96C69E010EC96EFF0ED3
:106720009EB602D0E82EFCD786EC31F075EC31F045
:106730009E96C69E910EC96EFF0E9EB602D0E82EA2
:10674000FCD79E96C69EA50EC96EFF0E9EB602D0C1
:10675000E82EFCD786EC31F0120075EC31F09E96F5
:10676000C69E26C0C9FFFF0E9EB602D0E82EFCD7FB
:106770009E96C69E810EC96EFF0E9EB602D0E82E72
:10678000FCD786EC31F0120075EC31F09E96C69E77
:1067900026C0C9FFFF0E9EB602D0E82EFCD79E96FB
:1067A000C69E010EC96EFF0E9EB602D0E82EFCD723
:1067B00086EC31F0120075EC31F09E96C69E910E7B
:1067C000C96EFF0E9EB602D0E82EFCD79E96C69EDE
:1067D000A50EC96EFF0E9EB602D0E82EFCD786EC41
:1067E00031F0120075EC31F09E96C69E910EC96E86
:1067F000FF0E9EB602D0E82EFCD79E96C69E000ED7
:10680000C96EFF0E9EB602D0E82EFCD786EC31F0A2
:1068100012000501256B266B276B286B899A400EA9
:10682000C76E200EC66E9E96C69E030EC96EFF0EE4
:106830009EB602D0E82EFCD79E96C69E27C5C9FFFD
:10684000FF0E9EB602D0E82EFCD79E96C69E26C5A9
:10685000C9FFFF0E9EB602D0E82EFCD79E96C69EBC
:1068600025C5C9FFFF0E9EB602D0E82EFCD79E9626
:10687000C69EC952FF0E9EB602D0E82EFCD7898A6A
:106880000F01C950FF0A01E1120005012E51130A40
:1068900005E005012E51170A0CE012000501F00E6B
:1068A000256FFF0E266F0F0E276F000E286F62EF09
:1068B00034F00501F00E256FFF0E266FFF0E276FD7
:1068C000000E286F899A400EC76E200EC66E9E96E7
:1068D000C69E030EC96EFF0E9EB602D0E82EFCD7F0
:1068E0009E96C69E27C5C9FFFF0E9EB602D0E82E13
:1068F000FCD79E96C69E26C5C9FFFF0E9EB602D047
:10690000E82EFCD79E96C69E25C5C9FFFF0E9EB6F3
:1069100002D0E82EFCD79E96C69EC952FF0E9EB6A8
:1069200002D0E82EFCD7898A0F01C950FF0A1DE06A
:1069300005012E51130A05E005012E51170A0BE03F
:1069400012000501000E256F000E266F100E276F36
:10695000000E286F12000501000E256F000E266F35
:10696000000E276F010E286F12000501256B266BA4
:10697000276B286B05012E51130A05E005012E51E6
:10698000170A0CE012000501000E216F000E226FA5
:10699000080E236F000E246FD7EF34F00501000EB0
:1069A000216F000E226F800E236F000E246F21C511
:1069B00000F122C501F123C502F124C503F125C56B
:1069C00004F126C505F127C506F128C507F12AEC13
:1069D0002EF000C125F501C126F502C127F503C13E
:1069E00028F5899A400EC76E200EC66E9E96C69EEA
:1069F000030EC96EFF0E9EB602D0E82EFCD79E96FF
:106A0000C69E27C5C9FFFF0E9EB602D0E82EFCD752
:106A10009E96C69E26C5C9FFFF0E9EB602D0E82EE2
:106A2000FCD79E96C69E25C5C9FFFF0E9EB602D016
:106A3000E82EFCD79E96C69EC952FF0E9EB602D087
:106A4000E82EFCD7898AC950FF0A08E104C125F560
:106A500005C126F506C127F507C128F5D89005011F
:106A600024332333223321332151F00B216F0501CD
:106A7000216742EF35F0226742EF35F0236742EF9E
:106A800035F02467D7EF34F00501100E2527E86AAA
:106A90002623E86A2723E86A28231200E86A05010A
:106AA0002E51130A06E005012E51170A0BE0020EC3
:106AB000120005012851000A03E12751F00B07E0FD
:106AC000010E120005012851000A01E0010E12001A
:106AD00029C500F12AC501F12BC502F12CC503F12E
:106AE00025C504F126C505F127C506F128C507F11E
:106AF000D9EC2FF003BF12004EEC35F0D8A4E0EF34
:106B000035F0899A400EC76E200EC66E9E96C69EC0
:106B1000060EC96EFF0E9EB602D0E82EFCD7898AFB
:106B2000899A9E96C69E020EC96EFF0E9EB602D030
:106B3000E82EFCD79E96C69E27C5C9FFFF0E9EB6BF
:106B400002D0E82EFCD79E96C69E26C5C9FFFF0E32
:106B50009EB602D0E82EFCD79E96C69E25C5C9FFDC
:106B6000FF0E9EB602D0E82EFCD79E96C69E000E63
:106B7000C96EFF0E9EB602D0E82EFCD7898A899A8C
:106B80009E96C69E050EC96EFF0E9EB602D0E82EDA
:106B9000FCD79E96C69EC952FF0E9EB602D0E82E26
:106BA000FCD7C9B0C9EF35F0898A0501100E252739
:106BB000E86A2623E86A2723E86A282368EF35F085
:106BC0001200899A400EC76E200EC66E9E96C69E13
:106BD000060EC96EFF0E9EB602D0E82EFCD7898A3B
:106BE000899A9E96C69EC70EC96EFF0E9EB602D0AB
:106BF000E82EFCD7898A0501256B266B276B286B4D
:106C00001200899A400EC76E200EC66E9E96C69ED2
:106C1000050EC96EFF0E9EB602D0E82EFCD79E96DA
:106C2000C69EC952FF0E9EB602D0E82EFCD7C9CF31
:106C300037F5898A1200899A400EC76E200EC66EFB
:106C40009E96C69EB90EC96EFF0E9EB602D0E82E65
:106C5000FCD7898A1200899A400EC76E200EC66E34
:106C60009E96C69EAB0EC96EFF0E9EB602D0E82E53
:106C7000FCD7898AFF0EE82EFED712004EEC35F0C5
:106C8000D8A41200899A400EC76E200EC66E9E963A
:106C9000C69E030EC96EFF0E9EB602D0E82EFCD72C
:106CA0009E96C69E27C5C9FFFF0E9EB602D0E82E4F
:106CB000FCD79E96C69E26C5C9FFFF0E9EB602D083
:106CC000E82EFCD79E96C69E25C5C9FFFF0E9EB630
:106CD00002D0E82EFCD79E96C69EC952FF0E9EB6E5
:106CE00002D0E82EFCD7898A0F01C950FF0AD8A428
:106CF000BDEF37F00501FE0E376F0501FF0E536F34
:106D0000FF0E546FFF0E556FFF0E566F15A6379985
:106D100015868FEC31F0AFC538F5B0C539F5B1C582
:106D20003AF5B2C53BF5B3C53CF5B4C53DF5B5C5BF
:106D30003EF50784BAC166F1BBC167F1BCC168F119
:106D4000BDC169F14BC14FF14CC150F14DC151F181
:106D50004EC152F157C159F158C15AF100011650B4
:106D6000010AD8B4C2EF36F000011650020AD8B4B6
:106D7000E7EF36F000011650040AD8B40CEF37F0F4
:106D8000BDEF37F00501476B486B496B4A6B050156
:106D90004B6B4C6B4D6B4E6B05014F6B506B516BDE
:106DA000526B8BA0379B71EC22F000C1DAF101C16C
:106DB000DBF102C1DCF103C1DDF100C13FF501C12E
:106DC00040F502C141F503C142F52BEF37F0050153
:106DD000476B486B496B4A6B05014B6B4C6B4D6BBA
:106DE0004E6B05014F6B506B516B526B71EC22F087
:106DF00000C1DAF101C1DBF102C1DCF103C1DDF157
:106E00006EEC23F000C147F501C148F502C149F518
:106E100003C14AF5BDEF37F0379BDAC13FF5DBC15F
:106E200040F5DCC141F5DDC142F571EC22F000C155
:106E30004BF501C14CF502C14DF503C14EF56EECA9
:106E400023F000C14FF501C150F502C151F503C156
:106E500052F52BEF37F00501616736EF37F06267C7
:106E600036EF37F0636736EF37F064673AEF37F0A5
:106E70004FEF37F0DAC100F1DBC101F1DCC102F103
:106E8000DDC103F161C504F162C505F163C506F119
:106E900064C507F1D9EC2FF003BFBDEF37F059C13E
:106EA00043F55AC144F5B9C545F50501110E326FD8
:106EB000899A400EC76E200EC66E9E96C69E060E1E
:106EC000C96EFF0E9EB602D0E82EFCD7898A899A39
:106ED0009E96C69E020EC96EFF0E9EB602D0E82E8A
:106EE000FCD79E96C69E27C5C9FFFF0E9EB602D050
:106EF000E82EFCD79E96C69E26C5C9FFFF0E9EB6FD
:106F000002D0E82EFCD79E96C69E25C5C9FFFF0E6F
:106F10009EB602D0E82EFCD725EE37F0322F02D0F5
:106F20009DEF37F09E96C69EDECFC9FFFF0E9EB640
:106F300002D0E82EFCD78EEF37F0898A899A9E9688
:106F4000C69E050EC96EFF0E9EB602D0E82EFCD777
:106F50009E96C69EC952FF0E9EB602D0E82EFCD762
:106F6000C9B0A8EF37F0898A0501100E2527E86A15
:106F70002623E86A2723E86A28231590079412003D
:106F800021C500F122C501F123C502F124C503F199
:106F9000899A400EC76E200EC66E9E96C69E0B0E38
:106FA000C96EFF0E9EB602D0E82EFCD79E96C69EF6
:106FB00002C1C9FFFF0E9EB602D0E82EFCD79E96F6
:106FC000C69E01C1C9FFFF0E9EB602D0E82EFCD7B7
:106FD0009E96C69E00C1C9FFFF0E9EB602D0E82E47
:106FE000FCD79E96C69EC952FF0E9EB602D0E82ED2
:106FF000FCD725EE37F00501100E326F9E96C69E27
:10700000C952FF0E9EB602D0E82EFCD7C9CFDEFFD4
:10701000322FFEEF37F0898A1200899A400EC76E30
:10702000200EC66E9E96C69E900EC96EFF0E9EB630
:1070300002D0E82EFCD79E96C69E000EC96EFF0EAB
:107040009EB602D0E82EFCD79E96C69E000EC96E54
:10705000FF0E9EB602D0E82EFCD79E96C69E000E6E
:10706000C96EFF0E9EB602D0E82EFCD79E96C69E35
:10707000C952FF0E9EB602D0E82EFCD7C9CF2DF51F
:107080009E96C69EC952FF0E9EB602D0E82EFCD731
:10709000C9CF2EF5898A12008FEC31F005012F51EE
:1070A000010A5FE005012F51020A16E005012F5188
:1070B000030A19E005012F51040A24E005012F51AC
:1070C000050A2BE005012F51060A39E005012F5171
:1070D000070A3FE0B1EF38F0602FAFEF38F05FC53F
:1070E00060F5B1EF38F0B0C500F101010F0E0017E7
:1070F00001010051000A35E001010051050A31E0AB
:10710000AFEF38F0B0C500F101010F0E001701011B
:107110000051000A26E0AFEF38F00501B051000A37
:1071200020E00501B051150A1CE00501B051300AFC
:1071300018E00501B051450A14E0AFEF38F0050141
:10714000B051000A0EE00501B051300A0AE0AFEF7D
:1071500038F00501B051000A04E0AFEF38F01590A7
:107160001200158012008B90A5EC2EF0B9C5E8FF37
:10717000D70802E3A5EC2EF0B9C5E8FFC80802E382
:10718000A5EC2EF0B9C5E8FFB90802E3A5EC2EF096
:10719000B9C5E8FFAA0802E3A5EC2EF0B9C5E8FFDF
:1071A0009B0802E3A5EC2EF01BEC36F0F29CF29E5D
:1071B0008B94C69AC2909482948C720ED36ED3A490
:1071C000FED789968A909390F29AF2949D909E9021
:1071D0009D929E92F298F29235EC33F0FF0EE8CF3A
:1071E00000F0E82EFED7002EFCD7F290F2868150F8
:1071F00081A8FDEF38F0F29E0300700ED36EF29678
:0E720000F29015840380C6EC2EF09AEF0BF08E
:10BF0000E844F926000C160C2B0C3F0C520C640C68
:10BF1000760C860C960CA50CB30CC10CCF0CDC0C6B
:06BF2000E80CF40C000C1B
:0200000400F00A
:0100C800FE39
:00000001FF
